:040000006F00204429
:100004000000000000000000480200004A02000056
:100014000000000040040000000000000000000098
:100024004004000040040000000000000000000044
:10003400B2180000000000004004000000000000AE
:10004400400400004004000040040000400400009C
:10005400400400004004000040040000400400008C
:100064004814000040040000400400004004000064
:10007400400400004004000040040000400400006C
:10008400400400004004000040040000400400005C
:10009400400400004004000040040000400400004C
:1000A40040040000C01800004004000040040000A8
:1000B40088180000D8170000400400004004000025
:1000C400400400004004000040040000400400001C
:1000D4004004000040040000400400004C170000ED
:1000E40040040000400400004004000040040000FC
:1000F4004004000092170000400400004004000087
:1001040040040000400400004004000040040000DB
:100114004004000000000000000000000000000097
:1001240000000000000000000000000000000000CB
:0C013400000000000000000000000000BF
:10014000397101436EC619A0397141536AC866CA34
:1001500062CC5ECE19A0397101535AD056D252D416
:100160004ED64AD826DA22DC06DE3301614082828E
:1001700041114AC026C222C406C68282B24D410144
:10018000024D924C224CB24B4101024B924A224A00
:10019000B2494101024992442244B2404101828065
:1001A0003D432A876373C3029377F700BDEFADE544
:1001B000937606FF3D8ABA960CC34CC30CC74CC756
:1001C0004107E36BD7FE11E28280B306C3408A0683
:1001D0009702000096966780A6002307B700A30643
:1001E000B7002306B700A305B7002305B700A30493
:1001F000B7002304B700A303B7002303B700A3028B
:10020000B7002302B700A301B7002301B700A30082
:10021000B7002300B700828093F5F50F9396850011
:10022000D58D93960501D58D61B7939627009702DA
:10023000000096968682E78086FA9680C1171D8F09
:100240003E96E374C3F8A5B701A001A0EFF25FF2F8
:100250000545EF00701F9922EF10207C7165130592
:100260000520EF10F000B707002083A507163775AB
:100270000000130585EBEF5030190925AA85377565
:100280000000130585ECEF503018EF30A00AEF3076
:100290000005014501B7EFF2BFED371402401C40E5
:1002A0003707FF08411193E717001CC05C40F98F26
:1002B0005CC01C403707F7FE6D17F98F1CC01C404F
:1002C0003707FCFF7D17F98F1CC05C40370701FF23
:1002D0007D17F98F5CC0B7079F001CC4EF00C07D7D
:1002E00002C402C6B7270240054798C31C404167B5
:1002F000B7160240D98F1CC03706020005679C4222
:10030000F18F3EC6A24785073EC4B24781E7A247A8
:10031000E397E7FEB71702409C431397E700635744
:10032000070685473EC6324785476313F706B7176A
:100330000240D843B706C1FFFD16D8C3D843D8C37F
:10034000D84313670740D8C3D843758FD8C3D84361
:10035000B7061100558FD8C39843B7060001558FD3
:1003600098C3984393166700E3DD06FED843B7169B
:100370000240719BD8C3D84313672700D8C32147D5
:10038000DC42B18BE39EE7FE410129B502C661BFA5
:10039000372702401C43F19B1CC3FDB7B716024030
:1003A000DC42370700201146B18B13070716638F15
:1003B000C70221466381C70495EB9C42918B9DC780
:1003C000B7470F00938707241CC3B7170240DC43CD
:1003D000918393F6F700B707002093870700B6973D
:1003E00094231C43B3D7D7001CC38280B7177A006D
:1003F00093870720D1BFDC42D4424166C983BD8BBD
:10040000F18E890745466393C700C94781EEB74619
:10041000024083A60680C18A89CEB7167A009386E9
:10042000062021A8B7160240D4421396E600E356F0
:1004300006FEB7163D0093860690B387D70269B7CC
:1004400001A0970100209381E15117510020130171
:1004500061BB17750000130525459705002093859E
:1004600065BA1386018263FAC5008322050023A0C2
:10047000550011059105E3EAC5FE138501829385B8
:1004800081B56377B500232005001105E36DB5FE46
:10049000FD42739002BC8D427390428093028008AB
:1004A0007390023097020000938202B693E232000A
:1004B00073905230EFF03FDE97020000938242D9F2
:1004C0007390123473002030B727014093870740A0
:1004D000631FF500EFF2DFC9854513050020EF002B
:1004E000B00E814513050020EF00100E65B182802B
:1004F0005C413707F1E01307F7EF944D7D8F9C4186
:10050000D58FD44DD58FD441A206D58FD98F5CC15C
:100510001C4537F7F1FF1307D77FD4457D8F9C49E2
:10052000D58F94458606D58FD98F1CC55C55370766
:1005300010FF7D177D8FDC29FD1793F7F70FD2078A
:10054000D98F5CD582801C4589C593E717001CC5EF
:100550008280F99BEDBF1C4593E787001CC5828014
:1005600008450D81058982801C4593E747001CC51D
:10057000828008450981058982801C4591C537071D
:100580005000D98F1CC582803707B0FF7D17F98FC7
:10059000D5BFA54763F7B7048D47138765FF3307BA
:1005A000F7020328C5009D47B397E70093C7F7FFFD
:1005B000B3F70701B396E600DD8E54C5994763E3B0
:1005C000C70495477D163306F6025859FD47B39781
:1005D000C70093C7F7FFF98F3396C5005D8E50D9DA
:1005E00082800D473387E502032805019D47B397B5
:1005F000E70093C7F7FFB3F70701B396E600DD8E78
:1006000014C96DBFB14763E2C7029547651633064B
:10061000F6021859FD47B397C70093C7F7FFF98F44
:100620003396C5005D8E10D9828095474D163306EE
:10063000F6025855FD47B397C70093C7F7FFF98FE8
:10064000B395C500DD8D4CD582806845420541815A
:10065000828008416D8D3335A00082805C4191C558
:1006600037070004D98F5CC18280370700FC7D17F3
:10067000F98FD5BF3C4989C593E707083CC98280FB
:1006800093F7F7F7E5BF3C4989C593E707043CC9F1
:10069000828093F7F7FBE5BF3C4993F7F7FD3CC930
:1006A0003C49DD8D2CC98280EFF29FACB7066745CF
:1006B000B7270240938636123797EFCDD4C313077E
:1006C000B79AD8C3D4D3011198C7D45B1387470313
:1006D00013962600E34B06FED45737250140130539
:1006E000054093E60620D4D7DC5BB7060020D58F03
:1006F0001CC31C431C4537070E00D98F1CC51C4565
:1007000093E717001CC53C4993E707043CC91C4507
:1007100093E787001CC52A842285993575FD372506
:100720000140832785401305054093E747001CC51A
:100730002A8422853D3D75FD372501400546C94582
:10074000814613050540B1352546230401003727AE
:100750000140B70550001C84637FF60423040100A8
:10076000A54621461C8463FFF606231501002304D9
:10077000010095461C8463F1F60E38853C85994648
:100780000D46B3F7D7020565130505803357D70229
:10079000B3D7C702BA97C207C1837C85B727014088
:1007A00003A78740799B23A4E7403C8505611D8D05
:1007B00042054185C5B283278740CD8F2324F7406A
:1007C00083270740898BEDDF1C848326C7440810EC
:1007D0008607AA972396D7FE1C84850793F7F70F01
:1007E0005C8495BFA30401009C846378F6001C849C
:1007F000850793F7F70F5C84B5B798849C840C1039
:100800000607850786072E97AE970357C7FE83D73F
:10081000C7FE63FDE7029C848607AE9783D7C7FEB9
:100820007C859C84988485078607AE9783D5C7FE10
:10083000931717001810BA972396B7FE9C84388533
:100840000C1085078607AE972396E7FE9C848507E4
:1008500093F7F70FDC8449BF1C8410103885890793
:100860008607B29783D7C7FEBA97C207C1837C8534
:100870001C84850793F7F70F5C84EDBD03A54182C7
:100880008280B70701401387074083A70740584B72
:10089000698F09C77D8D3335A00082800145828034
:1008A000B707014023AAA74082809C4513F70701A0
:1008B00013F8F70001C7D8413368E8008E2113F719
:1008C000F50F39C318418146854E3D4F930F800285
:1008D00093028004214E3396DE00B3F8C500631105
:1008E00016039398260033131F011343F3FF337746
:1008F000E300B318180133E7E800639FF70550C918
:100900008506E39AC6FD18C11307F00F6375B70497
:1009100054412146854E3D4F930F8002930280043F
:10092000414EB398CE0033F715016392E8021317D6
:10093000260001173313EF001343F3FFB376D30000
:100940003317E800D98E639DF701232A15010506A8
:10095000E319C6FD54C18280E39457FA10C94DB71C
:10096000E39757FE23281501DDB708456D8D333514
:10097000A000828048456D8D3335A00082800CC96F
:10098000828019C20CC982804CC98280370700C09E
:10099000B377E5006395E708370701405C4393565A
:1009A000B501584F9D8A9DE6F99BB70600FFFD16DD
:1009B000758F89C993160501C182D58FB706FF01CE
:1009C000758D498FB7060007D58FB7060140DCC289
:1009D000D8CE828005466396C600F59BB70680FF99
:1009E000F9B709466396C600ED9BB706E8FFC1B7A5
:1009F0000D466396C600DD9BB706FCFF4DBF114652
:100A00006397C60093F7F7F3B706C0FF4DB71546D7
:100A1000E391C6FA93F7F7CFB706E0FF49BF370770
:100A200000406391E702B7070140D84F4205B36722
:100A3000A70089E51345F5FFB377E50037070140C7
:100A40005CCF8280A9E337080140B7073000032656
:100A5000480013170501B376F50041836396F6024B
:100A6000B70600F9FD16B377D60003264800F18ECD
:100A70002322D80091C5558112053315A700C98FCF
:100A8000370701405CC382809317B50063D007022B
:100A90009357050193F6F7008D47B397D70093C797
:100AA000F7FFF18FB7060007D58FE9B793575501C8
:100AB0009207B317F700E5B7EFF28FEB37F4FF1F9C
:100AC000032744723706003E41119317970193465E
:100AD000F7FFF18F060737063E00718FD98F370673
:100AE000000113979600718FD98FBD824167F98EEF
:100AF000D58F02C202C402C623A4F18203578472B6
:100B000085452390E182032704721305D00323A6B1
:100B1000E1820327447023A2E1828D2C8327447055
:100B200037073A101307077093F7F7F06380E71061
:100B30006361F70237073210130707706380E70617
:100B400037073710130707706387E70841016FF015
:100B50006FE437073B1013070770638BE70A37070B
:100B60003D1013070770E393E7FE85452165393D86
:100B7000B7140140E177130480044C00138504800E
:100B80007C8222C61D3385679387C7334C0013854B
:100B900004C07C8222C6113BF9770DA085452165F2
:100BA000F533B7140140930700E0130480044C00B0
:100BB000138504C07C8222C6CD3989674C00371565
:100BC00001407C8222C6D5318D477C8222C64C00F2
:100BD0001385044025A8B7140140E1779387077077
:100BE000130480044C00138504807C8222C675396E
:100BF0009307D0E34C00138504C07C8222C6753174
:100C0000F9777C8222C64C003715014079393DBF07
:100C1000B7140140E177130480044C00138504806D
:100C20007C8222C65931930740208DB7B71401400A
:100C3000E177130480044C00138504807C8222C673
:100C4000AD318967F51799B723A8A182828003A7E0
:100C50000183854714216310F7021C31639CE7026E
:100C60003C21960793E707F837E700E093F7F70F83
:100C700036972300F740054793D756003317D70020
:100C8000544189CE938707048A07B7E600E0B697F8
:100C900098C38280EDF33C219607F9B79387070646
:100CA000E5B7B7160240DC423747FF7F7D17F98F63
:100CB0005D8DC8C28280371702405C439146B18B7C
:100CC000638CD706A146638ED706BDE71C43918B84
:100CD000A5C7B7470F00938707241CC137160240EA
:100CE0005C4237070020130707019183BD8BBA9739
:100CF00094231C41B3D7D7005CC15442A1829D8A82
:100D0000BA969422B3D6D70014C55442AD829D8AB8
:100D100036971423B3D6D70054C55842634C070006
:100D20005C42B98313F7370093874180BA979C23BD
:100D3000B3D7F6021CC98280B7177A0093870720C1
:100D400069BF5C435843C166C983BD8B758F8907F2
:100D5000C5466393D700C94701EF374702400327D1
:100D60000780418B09CF37177A001307072021A886
:100D70003717024058439316E700E3D606FE3717AD
:100D80003D0013070790B387E70281BF99C5371766
:100D900002401C4F5D8D08CF8280B7170240984FEC
:100DA0001345F5FF798D88CF828099C537170240AA
:100DB0005C4F5D8D48CF8280B7170240D84F1345F6
:100DC000F5FF798DC8CF828099C5371702405C47FF
:100DD0005D8D48C78280B7170240D8471345F5FF9D
:100DE000798DC8C782801A218D6793870704B62141
:100DF0007D8F9E21D58FD621D58FF621D58F962533
:100E0000D58FB625D58FD625D58FF625D58FD98FF9
:100E10001EA19E291EA982801E2189C593E7070471
:100E20001EA18280C207C18393F7F7FBC207C1836B
:100E3000C5BF4EA582804A2582800A256D8D333537
:100E4000A00082801E2137370140130707C0C20768
:100E5000C1836300E50237070040630CE500130718
:100E600007406308E5003717004013070780631643
:100E7000E500FA2193F7F7F8D98F9A2593F7F7CF82
:100E8000C207C183D98F371700401EA113070780FF
:100E90009C416310E5025CD5DE211EB5B7370140E9
:100EA000938707C06314F500BC251EB985475EA96A
:100EB0008280C207C1835EB5C5B71A31FD77FD17C1
:100EC000F98F1EB10358050256215E2D6577D22198
:100ED0001307F7CF7D8FF9772206FD17518FB3F7F0
:100EE0000701F22103D8A500C206420733660601B6
:100EF0003206D18F37360140C207130606C0C182C1
:100F00004183C183631AC50071767D16F18EF22587
:100F10001A06D18EC206C18256A1B71600405AAD3C
:100F20009386068098416315D50038C11EB1828032
:100F300042074183DDBF1E2189C593E717001EA12B
:100F40008280C207C183F99BC207C183CDBF83578B
:100F5000450491C52167D98F2312F5048280C60705
:100F6000C583DDBF5E2501C6DD8D4EA5828093C59C
:100F7000F5FFFD8DDDBF1E2189C593E707081EA182
:100F80008280C207C18393F7F7F7C207C183C5BF49
:100F90005A2DFD779387F77FF98FA205CD8FC20772
:100FA000C1835EAD8280B7170040938707806314CA
:100FB000F5002CC18280C205C181E5BFB717004092
:100FC000938707806314F500485182804A314205B7
:100FD000418182801E294A25ED8F4205418189C7C2
:100FE0006D8D3335A00082800145828093C5F5FF69
:100FF000C205C1810EA98280EFF28F971629F5777D
:10100000FD17F58FF621DA257971D58F1EA95625A2
:10101000FD779387379FF58FD6212A842EC6D58FEB
:101020009625D58FB625D58F5EA55E29C207C183CB
:1010300093F7F7CFD98F5EA96808B539B747014054
:1010400093870780B245631AF404A2575624654774
:10105000B387E702C206C186984163D20604060739
:1010600052244206B3D7E702130740064186B3D69F
:10107000E702B3F7E7029206635506028E079387ED
:101080002703B3D7E70213F77700B367D700C20788
:10109000C1831EA445616FF0EF8F925745BF0A07C9
:1010A000C1B7920793872703B3D7E702BD8BD58FCC
:1010B000F9BF91C55E250967D98F5EA582805A2543
:1010C000F977FD17F98FD5BF13F7F50F854715830E
:1010D000B395B7006319F7009307C500984301CE95
:1010E000D98D8CC38280894693074501E318D7FECA
:1010F00093070501E5B793C5F5FFF98DDDB793F5C6
:10110000F51F4EA182804A211375F51F82800A21A6
:101110006D8D3335A000828013F7F50F854615835A
:10112000B397B6006311D7025A25F98F1A210145EA
:101130004207418381CB0545A181B315B5006D8F71
:101140003335E000828089466314D7001A29F1BF45
:101150005A29E1BFEFF2CF81797113060002814570
:101160000808EFF0EF838545114502C202C402C6AC
:101170003139854513050020113901451D363715D4
:1011800001409307E00F4C00130505803724014010
:101190007C8202C6EFF06FF113050440EFF0CFB28E
:1011A00013050440EFF04FD0AA85239AA18237752A
:1011B0000000130585EDEF403025B7070E003ECE49
:1011C0000C088547130504402302F10202C802CA35
:1011D00002CC02D0EFF0CFB1854513050440EFF00B
:1011E0008FB6854513050440EFF0EFC9814513051F
:1011F0000440EFF0AFC613050440EFF0CFB5930401
:1012000004402685EFF0CFB56DFD1305044037246B
:101210000140EFF06FB5930404402685EFF06FB501
:101220006DFD37050080B53C130504408545EFF0A2
:101230006FC49305000213050440EFF0EFC545614C
:101240006FE05FF5EFE2DFF20111854521453D3E9C
:1012500085451165993E3714014085678D447C8032
:101260008A85C147130504C03EC426C2EFF0EFE3F0
:10127000130504C08565EFF08FF0896761498A85A1
:10128000130504C07C804AC426C2EFF00FE29167C8
:101290007C808A859147130504C03EC4EFF0EFE0DF
:1012A000E1778A85130504C07C804AC426C2EFF02A
:1012B000CFDFB70704013EC6B70702003EC8B70735
:1012C00000028507374400403ECAA1473ECC6C006F
:1012D0009D4713050480FC86393685451305048037
:1012E000253E05616FE01FEBEFE2FFE6B7440040EB
:1012F0002A891304900C9389048089454E85353ED4
:101300000DC5CA8513850480B74400401D361304FB
:10131000900C1389048085454A85053611CD1385C7
:101320000480113E1375F50F31A07D141374F40F72
:1013300069F401456FE07FE57D141374F40F61FCDF
:10134000CDBFEFE2FFE22A89371501402E84130555
:1013500005C08565B2840146EFF0AFE20D456937FF
:10136000135504011375F50F413713558400137598
:10137000F50F9D3F1375F40F853F0144931704014A
:10138000C18363EC97003715014005468565130559
:1013900005C0EFF00FDF6FE0FFDF1305F00FA93797
:1013A000B307890088A30504D1BFEFE27FDC4111B8
:1013B00085451145E13A930700107C8237150140BD
:1013C000C1473EC64C008D47130505803EC4EFF073
:1013D000CFCD41016FE01FDCEFE29FD94111854580
:1013E0004145EFF0BF9A8567938707807C82371568
:1013F0000140C1473EC64C008D47130505803EC4E1
:10140000EFF0AFCA41016FE0FFD8EFE27FD64111A4
:1014100085452145EFF09F97930700103714014051
:101420007C82C1473EC64C008D47130504C03EC4B4
:10143000EFF0AFC7054693050010130504C0EFF0A9
:101440004FD441016FE01FD54111114522C626C47A
:101450004AC2EFF00FC385476310F5043719014006
:10146000AA8401469145130509C0EFF08FD103C747
:10147000C1873E8409EF0545C923054691451305FB
:1014800009C0EFF00FD08947238EF18619A0E30C35
:1014900097FE1145EFF0CFC03244A24412494101FA
:1014A00073002030EFE2DFCC411185452145EFF09C
:1014B000FF8D85451145EFF05F8F930700203714AE
:1014C00001407C82E1473EC64C008D47130504C0B5
:1014D0003EC4EFF08FBD930700084C00130504C015
:1014E0007C82EFF08FBC41016FE0DFCAEFE25FC8A2
:1014F00001114D3F371400409307F01D8A851305F5
:1015000004803EC002C22314010023050100EFF055
:101510007F93130504808545B93CC167938707060F
:101520006C00130504803EC8231B010002C6EFF0C7
:10153000DF9813050480A145A13C1305048085456F
:10154000EFF07F9F854513050480EFF05FA00561F4
:101550006FE05FC4EFE2DFC1B7770000044103A989
:1015600007EF2A842685CA85EF30D03363580502F9
:1015700023202401B777000083A587EF0840EF30D0
:10158000303BEF40C0229315050137150040C18163
:1015900013050580EFF03FA16FE0DFBF2685EF4028
:1015A0004033B777000003A607F083A647F0EF208B
:1015B0008068E351A0FCB777000083A747EF1CC009
:1015C00055BFEFE2FFBA797137140140C1472A894C
:1015D000FC828D44C1474C08130504C03ECE26CC86
:1015E000EFF0AFAC0146130504C0C145EFF06FB991
:1015F00085452145EFF08FF9854537050800EFF067
:10160000CFFA8547FC824C08E147130504C026CC7D
:101610003ECEEFF08FA9894491474C08130504C0D2
:10162000E482375400403ECEEFF02FA80C10B707ED
:101630000C00130504C04AD03ED402D22316010286
:10164000EFF09F9B9307D0137C86680085473EC8C8
:101650004487EFF0CFDF0546130504C093055052D1
:10166000EFF09FA68545130504C0EFF09FA44561E8
:101670006FE05FB2EFE2DFAF79713714014093079B
:1016800000022A89FC828D44C1474C08130504C01E
:101690003ECE26CCEFF06FA10146130504C09305A2
:1016A0000002EFF00FAE85452145EFF02FEE8545A6
:1016B00037050400EFF06FEF93070040FC824C0801
:1016C000E147130504C026CC3ECEEFF00F9E8567A0
:1016D00093870780FC824C089147130504C03ECED7
:1016E00037540040EFF06F9C0C10B7070C00130547
:1016F00004804AD03ED402D223160102EFF0DF8FDD
:10170000930770137C8685475C87680085473EC8D1
:10171000EFF0EFD305461305048093055052EFF028
:10172000BF9A854513050480EFF0BF9845616FE0CF
:101730007FA6EFE2FFA32A84EFF07F9C93050008C9
:101740002285EFF0DF9C7DD96FE0DFA4411122C636
:10175000375400409305505213050480EFF0DF9B8F
:101760000DC513050480EFF01F9A9375F50F238CB8
:10177000B18203A541881C4D104954498507B3E740
:10178000C7026384D7003105052C32444101730040
:101790002030411122C637540040930550521305A2
:1017A00004C0EFF07F970DC5130504C0EFF0BF959F
:1017B0009375F50F238EB18203A581881C4D1049C6
:1017C00054498507B3E7C7026384D7003105ED228A
:1017D0003244410173002030411122C637040040D9
:1017E000854513050440EFF0EFFE01C9854513055B
:1017F0000440EFF0AFFFEF0050313244410173007D
:101800002030EFE2FF9601112E84AA84854505451C
:10181000EFF0AFD94C083705004026CAE084231EFC
:101820000100231D0100EFF0EFE105468545370576
:101830000040EFF02FF39307C0027C868D475C8752
:10184000680085473EC8EFF08FC0854537050040EA
:10185000EFF06FEE05616FE0FF93EFE27F91B70766
:10186000002083A50716896793870771B3D5F50212
:10187000A9473305F502FD15C205C1817D15420555
:10188000418141376FE01F91854537050040EFF0FA
:101890006FF411CD854537050040EFF02FF5CD20D1
:1018A00083C6C18705476394E600238E01867300D3
:1018B0002030B7F700E023A20700D92073002030C2
:1018C000411122C6373401408545130504C0EFF0AD
:1018D0006FF001CD130504C08545EFF02FF137758A
:1018E0000000130585F0EF4060433244410173006E
:1018F00020301DC9B296C206C18252A136A10CC5C4
:1019000009EE85471CA183A601849387018436874D
:1019100001EB54C588C30145828023000500E5B76B
:101920006306A7005847EDB77D5582800545828044
:101930000DC583A701841387018499E3054582803F
:10194000D4476396A6005845D8C701458280639462
:10195000A70014C3DDBFB687CDB77D558280EFE207
:101960003F8103A4018475DC1C2093F7F70F99C70E
:101970005E2099C3230004001C4482974044E5B7CD
:1019800083A70184054691E38280D62381CEBA23C2
:101990007D1742074183BAA3BA234207418319E363
:1019A00090A3B6A3DC47C5B7232605000CC150C1E0
:1019B00023240500054582805C4554411845850770
:1019C000B3E7D702638EE70058451C41BA978CA352
:1019D0005C4558418507B3E7E7025CC50545828051
:1019E0007955828018455C45630FF70018451C4106
:1019F000BA979C239CA11C4558418507B3E7E70291
:101A00001CC505458280014582805C4518454841DA
:101A1000998FAA9733E5A7028280B707002083A792
:101A200007160967130707F4B3D7E702C207C18394
:101A30002393F1842392F1848280B7F700E0D843A6
:101A40008146799BD8C303D741843306A70290CB44
:101A5000D4CB98431367070198C3984313671702C1
:101A600098C3D843058B75DF9843799B98C38280D0
:101A7000EFE20FF02A841165011185451105EFF0A1
:101A8000EFB0930700207C82371501408D473EC49C
:101A90004C00E147130505803EC6EFE01FE122C878
:101AA00037440140B70708000C08130504803ECCFA
:101AB00002CA231E0100EFF02FD4854513050480D0
:101AC000EFF02FDF05616FE0EFECEFE2CFE8B74416
:101AD0000140AE8932890144938404806345240126
:101AE0004A856FE08FEA930500042685EFF02FE228
:101AF0007DD9B38789008385070026850504C20543
:101B0000C181EFF0CFDFD9BF138781801C4393865B
:101B100081B53E95636BD500B7560020938606804D
:101B200063E5A60008C33E858280FD57EDBFEFE266
:101B30002FE437240140AA85954605461305044045
:101B4000EFE03FA5854513050440EFE01FA3930494
:101B5000044089452685EFE0DFAF65DD13050440CD
:101B6000EFE0BFAE6FE00FE30397418381472A9711
:101B7000634F070009CD05669306F6FFB6876358E5
:101B8000C700AA876305D50093170701C1833E8567
:101B90008280EFE2EFDD0545593F42054185E93797
:101BA000EF305046B777000083A587F1EF30001C77
:101BB000EF303052B777000003A607F283A647F252
:101BC000EF20A01DB777000003A687F283A6C7F217
:101BD000EF20A01CEF30B05A6FE0CFDBEFE24FD91F
:101BE0000945B137420541854137EF30B041B777FC
:101BF000000083A587F1EF306017EF30904DB77785
:101C0000000003A607F283A647F2EF200019B7777A
:101C1000000003A607F483A647F4EF200018EF3076
:101C200010566FE02FD7EFE2AFD40D4509374205CC
:101C300041851D3FEF30103DB777000083A587F148
:101C4000EF30C012EF30F048B777000003A607F27C
:101C500083A647F2EF206014B777000003A687F24F
:101C600083A6C7F2EF206013EF3070516FE08FD280
:101C7000EFE20FD01145653D42054185F535EF3066
:101C80007038B777000083A587F1EF30200EEF3072
:101C90005044B777000003A607F283A647F2EF206F
:101CA000C00FB777000003A607F483A647F4EF2020
:101CB000C00EEF30D04C6FE0EFCDEFE26FCB1945A7
:101CC000BD35420541854D359D67938787F40147B2
:101CD0009306100F92236369C5023A85EF20504B9B
:101CE000B777000003A607F383A647F3EF20E00AC7
:101CF000B777000003A687F383A6C7F3EF206055EC
:101D0000EF30F0476FE00FC905078907E314D7FCF0
:101D100013050000C5BFEFE2AFC579714800130697
:101D2000A0028145EFF0EFE11882930730053705F7
:101D300000206317F70298829307C0046312F7022A
:101D40000347D102D947631DF7001306A0024C00D8
:101D500013050502EF303060054545616FE08FC324
:101D6000B707002003C7C704130505029387C704FC
:101D700018A1983318B1B82338A1B83338B1D82393
:101D800058A1D83358B1F82378A1F83378B19827FF
:101D9000DC3718A5A304F5020145C1B7EFE24FBD3A
:101DA00041112A8940000408029908C01104E31D6A
:101DB00094FE1244A2442285A685EF304026635447
:101DC000A00026C222C41244B2452285EF3020254D
:101DD0006359A000A2452285EF30C02C6353050053
:101DE00022C4224541016FE0EFBAEFE2CFB64111C4
:101DF0002AC637250000130505C74D37B245AA8905
:101E0000EF30405CB777000083A5C7199384C18089
:101E1000EF300032B777000083A5C7182A894E85B6
:101E2000EF300031AA854A85EF20B03D8C40EF208D
:101E3000503D88C01385C180EFF0CFF141016FE0C4
:101E4000CFB4EFE24FB193874189F827C03722071B
:101E5000418FE0371389C1804204418F802B620497
:101E6000598CA285EF300056B777000083A507197B
:101E7000EF30002CB777000083A54719AA89228587
:101E8000EF30002BAA854E85EF20B037832509005F
:101E9000EF2030372320A9001385C180EFF08FEBAE
:101EA0006FE0AFAEEFE22FAB93874189B82B803B59
:101EB0002207418FA03B1389C1804204418FC02B70
:101EC0006204598CA285EF30E04FB777000083A5FC
:101ED000C719EF30E025B777000083A58718AA89D6
:101EE0002285EF30E024AA854E85EF2090318325AE
:101EF0000900EF2010312320A9001385C180EFF0E5
:101F00006FE56FE08FA8EFE20FA513874189834744
:101F10004702834637021147A207D58FFD17C20734
:101F2000C1836360F7021D678A071307C712BA9758
:101F30009C43138441898287B777000003A58714E7
:101F400095376FE08FA4B777000003A5C714713DE4
:101F5000CDBFB777000003A50715E535DDB71387BB
:101F600001811C239384018685C3B70600209386D4
:101F70000602BC2E903E9306800CA207D18FB38739
:101F8000D702230007009CC0371500408145130588
:101F90000580EFF04F819387C185984394400507F2
:101FA00098C3E310D7FA23A00700B777000003A572
:101FB0000715413D8D47A301F4022302040251B7E6
:101FC00013891181834709009384418585C7B70729
:101FD000002093870702E83B9C2FA2075D8DEF301E
:101FE0007002B777000083A54714EF20305888C0EF
:101FF000230009008840B13583C7D187B9F33C2855
:10200000034914014438A207B3E727010349340107
:102010004209B367F9000349440162093369F900D1
:102020007C284A85A207C58F6438C204C58F042C5A
:10203000E204DD8CA685EF30E038EF309009B77709
:10204000000003AA871583AAC7155286D686EF100B
:102050007049635E0500CA852685EF30A036EF30F3
:1020600050075286D686EF10F047E34C05ECB77761
:10207000000003A5C714953B894735BFEFE2CF8C1D
:10208000938421819C2093898185ADCB37040020E6
:10209000130404027C24483437790000A2075D8DC4
:1020A000EF30407683254914EF20504C23A4A184BF
:1020B0001C286834A2075D8DEF30C0748325491455
:1020C000EF20D04A23A6A1843C280838A2075D8DC2
:1020D000EF30407383254914EF20504923A8A18491
:1020E0007C284838A2075D8DEF30C07183254914E4
:1020F000EF20D04723A0A9002380040093874189C3
:10210000F82BC43B03C917012207458FE43BAC2FD2
:1021100003A50900C204458F842FA20513844189B9
:10212000E204D98CB82B22073367270103C9370192
:1021300042093367E90003C9470162093369E900CD
:10214000983FD98DB83F42074D8FCC2FE205D98DEE
:10215000EF20F06C635BA004CA852685EF20306C0D
:1021600063520502A6854A85EF30C025EF306076C0
:10217000B777000003A6871683A6C716EF10903620
:1021800063550502A301040223020402EF00304A52
:10219000B735000081461306803E9385E5F413852C
:1021A0000193EFF00FF56FD0BFFDA6854A85EF30A4
:1021B0006021EF300072B777000003AA071783AAE7
:1021C00047175286D686EF10F031635E0500CA8548
:1021D0002685EF30201FEF30C06F5286D686EF1075
:1021E0007030634805047C244434A207C58F6434EE
:1021F000C204C58F0428E204DD8CB777000083A5F4
:1022000007162685EF20106A63450502B7770000A0
:1022100083A547162685EF209060634CA000834974
:10222000440283473402A209B3E9F9009547639851
:10223000F9009547A301F40223020402ADB703AAF3
:10224000C1842685D285EF20905D6359A00003A547
:102250000185CA85EF20B05C6345A0009147639477
:10226000F9009147C1BF83A981842685EF3060665C
:102270002A8B4E85AE8BB77A0000EF30806503A6BF
:102280008A1783A6CA17EF1000285A86DE86EF1039
:102290007025635405025285EF30A06303A68A17A8
:1022A00083A6CA17EF10F07A2A86AE865A85DE8595
:1022B000EF1050238947E35FA0F6D2852685EF20F3
:1022C0001056635CA00203A50185EF308060B777EC
:1022D000000003A6071883A64718EF10C0222A8A19
:1022E0004A85AE8AEF30E05E2A86AE865285D68574
:1022F000EF10501F8D47E35FA0F2CE852685EF20BB
:10230000705AE35205EA854735B7EFD27FE63725A5
:102310000000130525B9EFF07FA813844189935776
:10232000850008B83CA893570501618148A8372566
:102330000000130565C23CB8EFF05FA69357850017
:1023400048B87CA893570501618108AC3725000087
:102350001305C5BD7CB8EFF07FA4935785007CA41E
:10236000935705017CB483C7D18748B4618108A81D
:1023700099E3EFF0BFD0EFF01FB96FD0BFE1EFD21C
:102380003FDF377500001306E0228545130545350C
:10239000EF3090079387418903C5370283C747020F
:1023A000A2075D8D6FD01FDFEFD29FDC3775000075
:1023B0001306202285451305052EEF30F00403A5F2
:1023C000418B2181420541816FD0DFDCEFD25FDAA2
:1023D0003775000013066021854513058531EF3000
:1023E000B00293874189D84F03C50702B777000031
:1023F00083A5473121836205598DEF207053EF305B
:10240000003B420541816FD0FFD8EFD27FD63775B0
:1024100000001306A020854513050538EF30C07E67
:1024200093874189984FC82FB777000083A547311C
:1024300021836205598DEF20B04FEF3040374205C0
:1024400041816FD03FD5EFD2BFD237750000130660
:10245000E01F85451305C52AEF30007B938741892E
:10246000D84B882FB777000083A5473121836205B9
:10247000598DEF20F04BEF308033420541816FD012
:102480007FD1EFD2FFCE377500001306201F8545A0
:102490001305C527EF30407793874189984BC82BA8
:1024A000B777000083A5473121836205598DEF205E
:1024B0003048EF30C02F420541816FD0BFCDEFD201
:1024C0003FCB377500001306601E85451305852434
:1024D000EF30807393874189D847882BB777000006
:1024E00083A5473121836205598DEF207044EF3079
:1024F000002C420541816FD0FFC9EFD27FC73775ED
:1025000000002E841306F01485451305051AEF30DC
:10251000A06F0547238FE1861385018F23820186F3
:10252000EFF00FC15C245834B7350000A207D98FF3
:1025300081461306803E9385051713850191239AE2
:10254000F188EFF00FBB6FD0FFC4EFD27FC223AA98
:10255000A18615470566B7350000238CE1868544C2
:102560008146130686BB938545021385018F23821E
:102570009186EFF00FB82388918E6FD0BFC1EFD254
:102580003FBFD425DC35A206DD8E954763FDD7001D
:10259000377500001306401285451305C51CEF3042
:1025A000A0666FD03FBFB425BC35A206DD8E930771
:1025B000002063FAD700377500001306B012854576
:1025C0001305C51FE9BF3775000013054523EF301C
:1025D000E074C1BFC16769768146FD170506139790
:1025E000060141836364B7003E8582803307D500CE
:1025F0001823B98F214713F8170085836305080056
:10260000B18FC207C1837D17420741836DF78506ED
:10261000F9B7EFD2FFB53715004013050580EFE09D
:10262000FF99EF306070EF3080759307100F3365BE
:10263000F502A94729053305F5026FD0BFB5EFD2E2
:102640009FB103A741882A84BE8405469305505252
:10265000631CA7043755004013050580EFE0DFA693
:102660002285EF007069131905010945EFF0EFBCF1
:102670002285EF00706883A74188931905011359DB
:10268000090193D90901014693055052375500407D
:102690006391870213050580EFE01FA333053941DD
:1026A0003335A0006FD07FAE37550040130505C00D
:1026B00075B7130505C0CDB7EFD29FAB3704002027
:1026C000834704024111130404025C801C3023156B
:1026D0000100AA84DC803C20AD450A855C813C3049
:1026E00023160100DC815C205C825C30DC827C2073
:1026F0005C837C30DC831C245C84930710FDDC84C9
:1027000085475C85EFF01FED93578500DC85834797
:1027100094024886DC86EFF0DFEFEFF00FB22685FB
:10272000EFF0FFF16DF93D468A852685EF001053E5
:1027300083A7418805469305505237550040639959
:10274000970013050580EFE03F9841016FD09FA4EB
:10275000130505C0CDBFEFD2BFA1370400208347CA
:1027600004024111130404025C801C302315010093
:10277000AA84DC803C20AD450A855C813C30231670
:102780000100DC815C205C825C30DC827C205C832C
:102790007C30DC831C245C84930700FDDC8485474B
:1027A0005C85EFF03FE393578500DC858347940217
:1027B0004886DC86EFF0FFE5EFF02FA82685EFF0E6
:1027C0001FE86DF93D468A852685EF00304983A7CD
:1027D000418805469305505237550040639997004C
:1027E00013050580EFE05F8E41016FD0BF9A13059E
:1027F00005C0CDBFEFD25F9503C9C500DC3501111F
:1028000022093369F9004209135909419314090156
:10281000C180954763FF970037750000A6861306B1
:10282000500C85451305C51CEF30003E05616FD087
:102830003F95B425BC35A206DD8E9307002063FAD0
:10284000D700377500001306B00C85451305C51F6A
:10285000E1BFAA8902CA02CC231E0100930A4101EA
:10286000368A370B0020B307DA40C207C18363E121
:10287000970C1384C18B1305C400130660028145B5
:10288000EFD01F923707002083470702A3052401DA
:10289000230504001CA0930707029433939A1400A5
:1028A0001309070214B0B42334A0B43334B0D423D2
:1028B00054A0D43354B0F42374A0F4339C2774B0E0
:1028C0001CA4930700031CB481471384818C63C547
:1028D000570993856400860593F5E50F1385C18B31
:1028E000EFF05FCF9317850021815D8D83479902BB
:1028F00056940AA03CA0EFF0DFD1EFF00F944E8584
:10290000EFF0FFD36DF913860A019385C18B4E85D5
:10291000EF00D03483A741880546930550523755C0
:102920000040639C370513050580EFE0EFF9FDBD1E
:102930001304CB08930B84031C40639947015C404C
:10294000014536C68297B2462390AA002104E3953A
:102950008BFE890A050A01BF101013F7E70F3297A3
:1029600013F61700B306F400035747FF11E2218363
:10297000850798A293F7F70F99BF130505C075B7A0
:10298000EFD26FFD370400201304C405AA89AE847A
:10299000328A1309040398341C406317F7005C4023
:1029A0005286A6854E8582972104E31624FF6FD0B8
:1029B000CFFDEFD2EFF841112A8CEF00F02F630822
:1029C000052A5145EFF06F871306200381451385D3
:1029D000C18B1384C18BB70D0020EFD06FFC8149F0
:1029E0008144014A930B1400B77C0000377D00003E
:1029F000138B0D026285EF003030630A0526628575
:102A0000EF00102D9387C18BD2973EC688A3930AFF
:102A10001A0089476384FA00638E0424182083C750
:102A20000D026314F710183083471B00631FF70E65
:102A3000377500001306102785451305C53BEF3099
:102A4000A01CA5476394FA0603D741898947631DF3
:102A5000F708382083472B00631BF708383083477B
:102A60003B006316F708582083474B006311F708B3
:102A7000583083475B00631CF706782083476B0060
:102A80006317F706783083477B006312F706182434
:102A900083478B00631DF704377500001306A028D9
:102AA00085451305853EEF30201621A08547E3EDCF
:102AB00097F8A9476385FA00894763FF970883D78A
:102AC0004189094714346392E7121307000363999D
:102AD000E606377500001306B02D854513058544BD
:102AE000EF308012C5498DA883C74186BDF383C7E7
:102AF000418195CB38303C20F98F5820F98F5830E0
:102B0000F98F7820F98F7830F98F1824F98F13070F
:102B1000F00F639AE700377500001306F02985452A
:102B20001305454149B791E085445286DE851385FA
:102B3000C18BEF30400293070003E3FD47EB05AA8A
:102B400041476398E602377500001306102E85454D
:102B50001305C546EF30400B1834C1476312F70C1C
:102B6000B54763FF570B8349D4008609C509568AC8
:102B7000D9B7138706031377F70F0546636DE60091
:102B8000377500001306802E854513050549EF3083
:102B9000A007B549D1B703C741811DCF1307000A6C
:102BA0001306E02E6389E6041307100A6398E60013
:102BB0001306402F854513054D4D1DB7268763F33A
:102BC000F40009479374F70F1306C02F854513854A
:102BD000CC4FEF30600391BF268763F3F4000947C1
:102BE0009374F70F13067030D5B79307000A639AF2
:102BF000F600130600313775000085451305054BB7
:102C000079B79307100A13066031E385F6FAA687B1
:102C100063F3E400894793F4F70F1306E0317DB7BF
:102C2000E3973AF59385DAFF93F5F50F1385C18B9A
:102C3000EFF05F9A330744018347E7FF0347F7FF4D
:102C4000A207D98F6397A700B2479823D947630A91
:102C5000F7000D47A68763F3E4008D4793F4F70F61
:102C6000E9B556869385C18B6285EFF07FD141012E
:102C70006FD0CFD0A547E39EFAE2F9B3EFD24FCFA2
:102C8000938701889843D566938606186307D70211
:102C9000050798C3371401408564938504801305A4
:102CA00004800546EFD0FFCD0146938504801305CF
:102CB0000480EFD01FCD6FD0EFCD23A00700B70762
:102CC000EFBE37E700E0938707083CC7E1B7EFD2D4
:102CD0002FCAB78400001385C486EF302004B7776D
:102CE000000083A5871903A5C18013844189EF20C3
:102CF0002044EF20B025AA85377500001305055242
:102D0000EF20907068245C343779000022055D8DD7
:102D10007C3483254914C207C98F082862055D8D5C
:102D2000EF200041EF209022AA853775000013059F
:102D30008553EF20706D28281C38832549142205FF
:102D40005D8D3C38C207C98F482862055D8DEF2034
:102D5000203EEF20B01FAA85377500001305C5542B
:102D6000EF20906A68285C388325491422055D8D20
:102D70007C38C207C98F082C62055D8DEF20403B6F
:102D8000EF20D01CAA853775000013050556EF20EB
:102D9000B067682C5C3C3777000022055D8D7C3C79
:102DA00083254731C207C98F0345040262055D8D43
:102DB000EF200038EF209019AA8537750000130521
:102DC0004557EF207064834724028345140237750A
:102DD0000000A207DD8D13054558EF20F062834700
:102DE00044028345340237750000A207DD8D1305C8
:102DF0008559EF2070611385C486EF203072938768
:102E000001879023371501409305001013361600F3
:102E10001305058090A3EFD0DFB66FD0AFB7EFD228
:102E20002FB503A58188EFF0DFB86FD0AFB6EFD232
:102E30002FB4371501400546A145130505C0EFD055
:102E40005FB43777000003274760370500408145AE
:102E50001305054023A6E180EFE0EF8D3715004014
:102E6000814513050580EFE00F946FD0AFB2EFD22C
:102E70002FB037050040854513050540EFE0AF8BC7
:102E8000371501409387418909470546930500108E
:102E9000130505C0A381E70223820702EFD07FAEAE
:102EA0006FD04FAFEFD22FAB1387A1871E231384B0
:102EB000A1878507C207C1831EA30547639AE70060
:102EC000371501400146A145130505C0EFD07FAB82
:102ED0001E201147636CF70037150040930540062C
:102EE00013050580EFE02F8C6FD02FAA1307600425
:102EF00093848186636BF70083A9040083A5C18056
:102F00004E85EF20C0116352A00293070000138585
:102F1000C1809CC023100400EFE0CFE31385019231
:102F2000EFE01FA1EFF0BFF4C1B74E85EF20701A9C
:102F3000B777000003A6875E83A6C75EE923EF206C
:102F4000102488C013858186EFE0CFE071BFEFD2F7
:102F50002FA2B704002093870402D42FB83FA20603
:102F6000D98E13873181102393840402938761865D
:102F700011C6230007001387D6FF9AA39A230507DB
:102F8000420741836305D7009AA36FD0AFA03725CE
:102F90000000130505C72390070037790000EFE014
:102FA000FFDF138441898325491413578500935704
:102FB000850138AC1357050138BC5CAC08BCEF2068
:102FC0002017EF20A078AA85377500001305055F4C
:102FD000EF2090433C2C183CA838A2075D8F3C3C66
:102FE000402CC207D98F62045D8CDC28A2075D8D5E
:102FF000EF20500183254914EF105057A285EF2090
:10300000600AE35405F8B735000081467946938598
:1030100045EA13850192EFE0DF8D13850193EFE020
:103020003F91A5B7EFD22F931387F1871C2301118E
:1030300093861700F51714A393F7F70F9306B00FB5
:1030400063EDF6001385018F2382018623000700BC
:10305000EFE01F8E05616FD04F9341468145130508
:10306000E100EFD0EF9337040020834704021304FC
:103070000402DD455C821C3048009384F187DC82C9
:10308000FD577C83FD573EC4E9779387F71F7C8605
:1030900083C78187DC8703C7518983C641899387AA
:1030A00041892207558FA308E100935687003820F5
:1030B0002308D1002309E1003830A309E10058209A
:1030C000230AE1005830A30AE1007820230BE10035
:1030D0007830A30BE1001824230CE1009837BC27BB
:1030E000A207D98F13D78700230DF100A30CE100AD
:1030F000EFF04FCE93578500A30DF1008347940264
:10310000230EA1002944A30EF100EFF08FD0EFE0D1
:10311000DF921389418703250900EFF04FD221E5A3
:103120009387E187942305476397E6002380070090
:103130002380040005B7032509006D464C00392E95
:103140000327090083A74188054693055052375548
:1031500000406317F70013050580EFD0FFF6DDBDD3
:10316000130505C0DDBF7D141374F40F59FCDDB5E4
:103170009387C1869043938641810506B705002059
:1031800090C3238006009385050203C7250203C56B
:1031900015022207498F631EE600EFC27FFD23A0C0
:1031A00007001385019185479CA2EFE06FF86FC07F
:1031B0007FFE8280EFC2DFFBB70700209387070204
:1031C000B8231384418938A0B833238A0188A38A9D
:1031D000018838B0D823372500001305C5BD58A095
:1031E000D8339384418958B0F82378A0F8339C27CA
:1031F00078B0370700201307C7041CA43C271437F6
:10320000A207D58F1CB4A1833CA45C273437A20746
:10321000D58F3CB4A1835CA4EFE05FB893578500E1
:1032200048B47CA493570501618108A837250000A4
:10323000130525B97CB4EFE07FB69357850008B835
:103240003CA893570501618148A837250000130564
:1032500065C23CB8EFE09FB49357850048B87CA89E
:1032600093570501618108AC37250000130505C798
:103270007CB8EFE0BFB29357850008BC3CAC9357D5
:103280000501618148AC372500001305A5CB3CBC86
:10329000EFE0DFB09357850048BC7CAC9357050145
:1032A00061817CBC2300A402371401409305001007
:1032B000130504C0EFD00FEC814701C991451305F8
:1032C00004C0EFD08FEAB337A000A380F4022381BB
:1032D0000402A3810402238204026FC0BFEBEFC289
:1032E0003FE9EFE05FA3EFF0FFECB7350000814668
:1032F0001306803E9385E5CC13850190EFE06FDFE8
:10330000B73500008146130640069385E5E1138535
:103310000194EFE00FDEB7350000F9461306803E5A
:103320009385C5C713850195EFE0AFDCEFE02FE390
:103330006FC05FE6EFC2DFE30545EFE00FD2B520D7
:10334000EFE0CF9AEFD01FE1EFE02F86EFE0CF88DC
:10335000EFD05FEFEFE06F8B1385C180EFE08F9FC1
:103360006FC05FE3EFC2DFE0014405C1002111CC73
:103370005C410D47639EE7003755004093F5F50F1C
:1033800013050580EFE0EFBA054422856FC09FE08A
:1033900011470544E39BE7FE3755004093F5F50FD1
:1033A000130505C0EFE0EFB8CDB7EFC27FDC3704FF
:1033B00000201304440C1306800C9385019613051A
:1033C000C400EFE06FDE08448544EFE0AFAA04A03C
:1033D0001306C012938581A21305840223A281885B
:1033E000EFE08FDC48507104EFE0AF9D04A0014591
:1033F00023A481886FC01FDAEFC29FD73715014021
:10340000054693050002130505C0EFD08FD76FC0A6
:103410007FD8EFC2FFD53715014001469305000262
:10342000130505C0EFD0EFD56FC0DFD6EFC25FD474
:10343000371501400546C145130505C0EFD06FD4CF
:103440006FC05FD5EFC2DFD2371501400146C145DD
:10345000130505C0EFD0EFD26FC0DFD3EFC2BFCFEF
:1034600003A741882A842E8AB28993844188631EE7
:10347000A700EFF07FF80149634039039C40639651
:103480008702EFF01FF96FC05FD083A78188E394B4
:10349000A7FEEFF0BFF9C5B7B3072A018385070080
:1034A00022850509EFF01FECC1BF83A78188E39C4B
:1034B00087FCEFF03FF9C1BF814709C91821814757
:1034C00011C75C49084D898FB337F0003E85828073
:1034D000EFC21FCA41112A84A3070100EFF0DFFDEC
:1034E00019C59305F1001305C400EFE0AFCF030544
:1034F000F10041016FC01FCAEFC29FC73105EFE065
:10350000CFD06FC03FC93708100001117D18337745
:10351000B80026CA3378D80093D4450113D34601A6
:10352000131E37004EC61357D5010E089357D60108
:1035300093F4F47F1373F37F06CE22CC4AC893D959
:10354000F50193DEF6013367C701131F350033E839
:103550000701931F3600338E64406380D919635688
:10356000C0136304031CB70680009307F07F336821
:10357000D800638FF4369307800363C0C735FD47D7
:1035800063CDC747130500023305C541B3D7CF014B
:10359000B316A8003399AF00DD8E33392001B3573D
:1035A000C80133E926011D8F33092F41B3372F019D
:1035B0003306F7409317860063D40724370780004B
:1035C0007D173374E600630C042C2285EF20C05174
:1035D000130785FF93070002998FB357F90033163D
:1035E000E400D18F3319E9006341972A33059740EE
:1035F000130615007D47634DC73813070002118F6E
:10360000B356C9003319E9003397E700558F3339B2
:1036100020013369270133D6C700814493777900AD
:1036200081CF1377F90091476308F700130749002A
:10363000333927014A963A899317860063D6071CC7
:10364000138514009307F07FCE856304F520B70738
:1036500080FFFD17F18F9398D70113593900A60702
:10366000B3E82801B1831375F57F9396C70052051F
:10367000F2406244B182FE05C98ECD8ED2444249E9
:10368000B2494685B68505618280631E0E0A1383A2
:1036900014001373E37F63170322B367E701B36872
:1036A000F801639D041A6387074063860844330961
:1036B000FF41B307074133362F013386C7409317C5
:1036C000860063D6074C3389EF41B307E84033B631
:1036D0002F013386C740F68991B76350C00F63004E
:1036E000030CB70680009307F07F3368D800638A25
:1036F000F43A9307800363CBC713FD4763DFC735F5
:1037000013090EFE93070002B3562801630AFE0058
:10371000130900043309C94133192801B3EF2F01FC
:103720003339F0013369D90031A2B367F801638AF4
:10373000071C9307FEFF638C07389306F07F63092D
:10374000DE1A3E8E0DBDB305934063910422B3672C
:10375000E701638707329387F5FF63810744930688
:10376000F07F638CD520BE859307800363CCB72A96
:10377000FD4763CFB73C930700028D8F3319F700E5
:10378000B356BF00B317FF003369D900B337F00059
:103790003357B7003369F9003308E84041ACB367E9
:1037A000F801638007349307FEFF638A07209306BE
:1037B000F07F6308DE2E3E8E2DBF631E0E149386AF
:1037C000140093F7E67F63910734B367E7016395CD
:1037D000042C6380073EB367F801638E073033091A
:1037E000FF01B3070701333FE9013386E701931770
:1037F000860063D70700B70780FFFD177D8E8544DD
:1038000093777900E39F07E09317D6019358390027
:10381000B3E8F800935736001307F07F638DE40494
:10382000B207B18313F5F47FCE8581B53369F80112
:10383000333920017A99B337E9013386E7009317CA
:103840008600E3DF07FA85049307F07F6396F41898
:10385000CE851305F07F8147814801BDC1EB6384AC
:10386000083A931636009317D8018D82B3E8D70033
:10387000F68993573800B3E7F800F9DB8145130563
:10388000F07FB70708008148CDB3370680FF7D166B
:103890007D8E93777900998CE39507D8B5B74A85E3
:1038A000EF20802413078501FD47E3D5E7D21306F7
:1038B00085FFB317C900014905BB3369F8013339E6
:1038C0002001DDB13309FF413306074133342F01B5
:1038D000330486409317840063CD0724B3688900BE
:1038E000E39308CE8147814981441DBFE39808F8DE
:1038F0000E059317D7010D81B3E8A7009357370042
:103900009DBF0E059317D7010D81B3E8A700F28480
:103910009357370011B73305934063820412B706FB
:1039200080009307F07F558F630DF32E930780037C
:1039300063CBA720FD4763C3A72A93070002898FA3
:103940003319F700B356AF00B317FF003369D9003E
:10395000B337F0003357A7003369F9003A987E99DE
:10396000B337F901338607019A84D1BDB7068000C9
:103970009307F07F558FE319F3DE931736008D839D
:103980009318D801B3E81701F68993573800E5B5C5
:10399000130715FE9306000233D7E700630AD6002B
:1039A000930600043386C6403396C7003369C900C6
:1039B000333920013369E9000146814491B5330967
:1039C000FF01B30707013336E9013E9693178600DE
:1039D0008544E3D707E28944B70780FFFD17F18FDD
:1039E0001357190013791900336927019398F701C8
:1039F00033E9280113D6170015B113090EFE9307FA
:103A00000002B3562801630AFE00130900043309BB
:103A1000C94133192801B3EF2F013339F00133695C
:103A2000D90059B63369E7013339200133892F4171
:103A3000B3B72F013306F8409A84F689A5BEB36761
:103A4000E701638207189307F5FF6384071C930659
:103A5000F07F6304D5123E85D1BD93070002B38782
:103A6000C741B316F8003399FF0033D6CF01D18E8A
:103A700033392001B357C80133E926013E975DBBB6
:103A8000931736008D839318D801B3E81701AE84DD
:103A900093573800F68949B3EDC33369F801E31F42
:103AA00009DC0E059317D7010D81B368F500935714
:103AB0003700D1B36381080E931636009317D801EF
:103AC0008D82B3E8D700F6899357380091BB33094C
:103AD000FF41B3070741333F2F013386E741854458
:103AE000D1BC0E059317D7010D81B368F500F284A0
:103AF0009357370015B30E059317D7010D81B3E81F
:103B0000A7009357370029BB9307F07FE382F6D4D1
:103B10003309FF013336E901B3070701B2979398E0
:103B2000F7011359190033E9280113D61700B68499
:103B3000C1B93389EF413307E84033B62F0133046D
:103B4000C740F68949B43369E7013339200101BD23
:103B5000938705FE93060002B357F700638AD500EA
:103B600093060004B385B6403317B700336FEF00F8
:103B70003339E0013369F90055BD931736008D8361
:103B80009318D801B3E8170193573800EDB1B36823
:103B9000C900E39708C68147814959B13389EF418C
:103BA000B307E84033B62F013386C740F689854412
:103BB00011B4931636009317D8018D82B3E8D7005D
:103BC00093573800B1B9931636009317D8018D82F8
:103BD000B3E8D700AA84935738003DB9930705FE90
:103BE00093060002B357F700630AD500930600045A
:103BF0003385A6403317A700336FEF003339E00158
:103C00003369F900A9BB81451305F07FB7070800A8
:103C1000A9BC3309FF01B30707013336F9013E960A
:103C200075B3931636009317D8018D82B3E8D70089
:103C30009357380089B113D74501B7071000FD1716
:103C400013D846011377F77F9308F07F33F3B7005B
:103C50002A8EF58FFD81B28E1378F87FFD8263087E
:103C60001703630018030DEBB368A3006314080087
:103C70005D8E29CA638508046388D502054595EDE4
:103C80008280B3E8C700E38008FE795582803365FF
:103C9000A30065FD630CE802631408005D8E79DE05
:103CA000E39ED5FCE34CE8FC63480701E3E867FCCE
:103CB0006303F302637FF30081E57D558280F5DEC7
:103CC000054582800145E39B08FA82805D8E69DAB2
:103CD0006DBF01458280E3E3CEFB0145E372DEFB6D
:103CE000E5F1E1BF13D74501B7071000FD1713D861
:103CF00046011377F77F9308F07F33FEB700AA8E53
:103D0000F58FFD81328F1378F87FFD82630E1703E4
:103D1000630D180129E3B368AE00631F08005D8ED0
:103D200001EE0143638C080421A8B3E8C7000943EE
:103D3000639608046DD305A0638408046385D502E7
:103D400005438DCD7D531DA8B368AE00094363972D
:103D50000802630AE802631408005D8E75D2E391DD
:103D6000D5FEE34FE8FC63490701E3EBC7FD630FB2
:103D7000FE0001436374FE00F1D505431A8582807D
:103D8000EDFE7D53E5BF5D8E79DACDBFE36ADFFBE3
:103D90000143E3F5EEFFF5F175B739714AD813D950
:103DA00045014ED652D456D29399C50006DE22DC88
:103DB00026DA5AD05ECE1379F97F2A8A93D9C900C0
:103DC00093DAF501630D090E9307F07F6306F91886
:103DD0001354D5018E09B36934013704800033E4EC
:103DE000890093143500130919C08149814B13D7F9
:103DF0004601139AC6001377F77FB285135ACA009B
:103E000013DBF601630B07109307F07F6303F704DE
:103E10009357D6010E0A33EA4701130717C0B707B5
:103E20008000B367FA00931536003A99814833C78A
:103E30006A01BD463A851308190063E8361717363C
:103E400000001306A67C8A09B29983A60900B296DF
:103E50008286B367CA001309F97F6399071293E951
:103E6000290081458948E1B701479307F07F37046E
:103E7000080081443204D20731807E075D8C598C62
:103E8000A285F250625426854259D254B259225A20
:103E9000925A025BF24B216182805A853E84AE8445
:103EA000C68B8947638DFB0E8D47E38FFBFA8547F1
:103EB0002A87639EFB3881470144814465BF33E410
:103EC000A90061C036C632C4638C092A4E85EF1042
:103ED000B0412246B246AA87130755FF7544938422
:103EE00087FF198CB399990033548A0033643401E5
:103EF000B3149A0013D746011309D0C0139AC60011
:103F00001377F77F3309F9408149814BB285135A02
:103F1000CA0013DBF601E31907EEB367CA00B1C7A5
:103F2000630F0A22528532C4EF10103C22462A87C2
:103F3000930655FFF547930587FF958F331ABA000F
:103F4000B357F600B3E74701B315B6003309E940AC
:103F50001309D9C08148E1BD33E4A90001ECA149AE
:103F600081441309F07F894B59B593E919008145C4
:103F7000854875BD4E84AA84B1491309F07F8D4BE5
:103F8000BDB5914981440149854B95B593E9390007
:103F9000D2878D4869BD89475685E397FBF02A870C
:103FA0009307F07F01448144F1B5C16E1386FEFF93
:103FB00093D6040113DE0501F18CF18D3386950251
:103FC0003383B6029358060133059E021A95AA98C8
:103FD000B382C60363F36800F692C16F1383FFFFD9
:103FE00033F5670093D30701B3F76800C207337353
:103FF00066003E933306950293D80801B387A60264
:10400000135F0601B3849302BE94FA94B38E7602D2
:1040100063F3F400FE9E416A9307FAFF935F040185
:10402000B376F400B3F9F4007D8EC1803384D502F9
:10403000C209338FD401B299CE98B307DE02935EE2
:104040000401B385BF02AE97BE9E330EFE0363F339
:10405000BE00529EC1679385F7FF33F6BE006D8C9C
:104060004206229693DE0E01B305D502769E338575
:10407000AF0213D40501B386D302AA96A296B38FDA
:10408000F30363F3A600BE9F41657D15B3F7A60059
:10409000C2076D8DAA97B3855800B3B93501FA9759
:1040A000B2953384370133B6C500B30EC4013385EE
:1040B000CE0033343401B3B7E701C18F33BECE0134
:1040C00013D406013336C5003E943366CE00939474
:1040D000950032947E94B3E46400260493567501EF
:1040E000B3349000DD8193179500CD8C558CDD8C19
:1040F0009317740063DB070093D714008588931629
:10410000F401DD8CD58C058042899307F93F635912
:10411000F00893F6740081CE93F6F400114663889C
:10412000C60093864400B3B496002694B6849316D2
:10413000740063D80600B70700FFFD177D8C930756
:1041400009409306E07F63CFF60E93D634009314B4
:10415000D4012604D58C318093F7F77F21BB3285BB
:1041600032C4EF10701893065501F147130705028A
:104170002246E3D1D7DC6115B317A6008145F9B318
:10418000EF10901613075501F145930705022246DB
:10419000B246E3D5E5D461153314AA00814499BB36
:1041A00085469D8EB1E71309E941B3972401B3D445
:1041B000D40033192401B337F000B3649900DD8CC7
:1041C00093F77400B356D40081CF93F7F4001146EF
:1041D0006388C70093874400B3B49700A696BE8453
:1041E0009397860063D8070485470144814459B1F9
:1041F00013068003E341D6CC7D46E356D6FA055636
:10420000B307F640930500023356F4006387B60007
:104210001309E943B3172401DD8CB3349000D18C2A
:1042200093F67400014499CA93F7F400114681464D
:10423000E392C7FA139496003180F6068D80D58CF0
:1042400081470DB99307F07F0144814425B142892C
:104250006DBD370710007D1701113373B70093D878
:104260004601758F935ED60122CC26CA0E0393D4E5
:1042700045019357D5010E0706CE4AC84EC693F89E
:10428000F87F130EF07F33E7EE0093F4F47F13D43E
:10429000F50133E36700131F3500FD82931E3600DE
:1042A0006380C81993C61600B38514416305D41200
:1042B0006351B018638B081AB70780005D8F638164
:1042C000C4599307800363C4B734FD4763C5B74837
:1042D000930700028D8FB3D9BE003318F700B39E49
:1042E000FE00336838013357B700B339D001336863
:1042F00038013303E340B3090F41B3373F013306BD
:10430000F3409317860063D30724370980007D1993
:1043100033792601630F092C4A85EF10E07C1307DF
:1043200085FF93070002998FB3D7F9003316E90090
:10433000D18FB399E9006344972A058F13061700BC
:10434000FD4663C5C63A13070002118FB3D6C900F4
:104350003398E9003397E700558F33380001B3698C
:10436000070133D6C700814493F7790081CF93F6D4
:10437000F90091476388F6009386490033B8360107
:104380004296B6899317860063D6071C13871400DC
:104390009307F07F05886306F720B70780FFFD17B6
:1043A000F18F1398D70193D93900A60733683801E4
:1043B000B1831377F77F9396C7005207B1827E04CB
:1043C000D98EC18EF2406244D2444249B2494285FC
:1043D000B685056182806356B00A638A0812B70702
:1043E00080005D8F6387C42D9307800363C7B71870
:1043F000FD4763D2B73C138805FE93070002B3590B
:104400000701638AF50093070004B385B7403317AB
:10441000B700B3EEEE003338D0013368380195A20F
:10442000B367D7019385148099E393C61600630A96
:10443000D404D1E19387140093F7E77F6399071EB3
:10444000B367E3013368D701639204166382073CC4
:1044500063160842131835009316D3011358380019
:1044600033E806019357330019A2B367D701638578
:10447000071A9387F5FF638B073A638CC523BE85C4
:1044800089B56399051C9386140093F7E67FC1EF05
:10449000B367E30163900436638D0744B367D701C4
:1044A000639407460E051318D3010D813368A800E5
:1044B000935733006DA8B385984063970420B36782
:1044C000E301638D07309387F5FF63890740130588
:1044D000F07F6383A520BE859307800363C2B72A5C
:1044E000FD4763C8B73C930700028D8F3318F30074
:1044F0003356BF00B317FF003368C800B339F0006C
:104500003353B3003368380133076740B5ACB36742
:10451000D701638307109387F5FF638F071E6380BE
:10452000C52FBE85D1B59307F07F638BF606FA9E43
:1045300033B6EE01B307E300B2971398F70193DEA9
:104540001E00B369D80113D61700B68493F779001B
:10455000E39F07E09317D60113D839003368F800BA
:10456000A685935736001307F07F6380E506B207F0
:10457000B18313F7F57F05883DBD3367D701333825
:10458000E000B309E801B3B7E90133866700931788
:104590008600E3DD07FA85049307F07F639CF41837
:1045A00005881307F07F8147014831B563910710F3
:1045B0006301083C131836009317D70113583800CD
:1045C0003368F800368493573700B367F800E9DBA7
:1045D00001441307F07FB70708000148E9BB37061D
:1045E00080FF7D167D8E93F77900998CE39107D833
:1045F00095B74E85EF10404F13078501FD47E3D275
:10460000E7D2130685FFB397C90081492DB33368FC
:10461000D70133380001C5B1131835009317D30102
:10462000135838003368F800935733002DBFB3098F
:10463000DF413309E34033363F013309C940931763
:10464000890063CA072033E82901E31508CC8147B4
:10465000014431BFB385984063810414B7068000DC
:104660009307F07F3363D3006381F82093078003BF
:1046700063CCB722FD4763C9B72C930700028D8F27
:104680003318F300B356BF00B317FF003368D800E8
:10469000B339F0003353B300336838011A97B309C4
:1046A000D801B3B7D9013386E700C684CDB5E3118D
:1046B00008F2131835009317D301135838003368E4
:1046C000F8009357330011B7370580009307F07F48
:1046D0003363A300E392F8E00E061318D7010D82AE
:1046E0003368C800935737003684C5B5051793065D
:1046F000000233D7E700630AD6009306000433862E
:10470000C6403396C700B3E9C90033383001B369F6
:10471000E800014681441DBDB309DF01B307E30092
:1047200033BFE9013386E701931786008544E3DF51
:1047300007E08944B70780FFFD17F18F13D71900F1
:1047400013F81900336807019399F701B3E90901D8
:1047500013D6170011B9138805FE93070002B35949
:104760000701638AF50093070004B385B740331748
:10477000B700B3EEEE003338D00133683801A5BE80
:104780003363E30133386000B3890E41B3B73E01B0
:104790003306F740C6843684ADB6B367E30163875A
:1047A00007189387F5FF638C071C9306F07F638ED1
:1047B000D50ABE8565BD930700028D8FB3D9BE00B3
:1047C0003318F700B39EFE00336838013357B70043
:1047D000B339D001336838013A9365B31318360002
:1047E0009317D7011358380033E8070136849357DD
:1047F000370095BBBDCB3367D701E31B07DC0E0544
:104800001318D3010D813368A8009357330075BB8B
:10481000E30F08E2131836009317D7011358380036
:104820003368F80036849357370091B3B309DF41FA
:10483000B307E340333F3F013386E7418544D1B4BA
:10484000131835009316D3011358380033E80601C6
:10485000935733009DBBB389EE413306674033B9AC
:104860003E0133092641368475B40E061318D7016C
:104870000D823368C8009357370081BBB309DF410D
:10488000B307E34033363F013386C74093178600B2
:1048900063D7070AB389EE41B3076740B3BE3E0151
:1048A0003386D7413684C9B43363E30133386000BB
:1048B000FDB3138805FE93070002B3590301638A11
:1048C000F50093070004B385B7403313B300336F8B
:1048D0006F003338E001336838017DB5B389EE41AC
:1048E000B3076740B3BE3E013386D7413684854463
:1048F00009BC131836009317D701135838003368D2
:10490000F80093573700A5B1B309DF01B307E300FF
:1049100033BFE9013386E70193178600E3D807C266
:10492000B70780FFFD177D8E85440DB10E06131865
:10493000D7010D823368C800935737002DB133E893
:10494000C900E30608D019B1138805FE93070002D9
:10495000B3590301638AF50093070004B385B74098
:104960003313B300336F6F003338E001336838011D
:104970003DB301441307F07FB70708002DBCB3090E
:10498000DF01B307E300B3BED9013386D70169BBAA
:10499000411106C622C426C20DCD9357F541B3C4BA
:1049A000A7009D8C2A842685EF1000149306E04111
:1049B000898EA9477D8093F6F67F63CDA7022D47A8
:1049C000098FB3D7E4005505B207B394A400B183AF
:1049D00029A00144814681478144B207D206B183B0
:1049E0007E04D58FC18FB24022442685BE85924475
:1049F000410182805515B397A400B207B183814469
:104A0000E9BF4111370780007D1713D8750126C211
:104A1000935475013373A70093F4F40FB376B70082
:104A20004AC01378F80F1359F50106C622C4FD8158
:104A30009A8726854A86131E3300939E3600B388D4
:104A40000441630AB90E6350100D63040814930700
:104A5000F00F638BF414B7070004B3EEFE00ED47CC
:104A600063C1172993070002B3871741B397FE006C
:104A7000B3D81E01B337F000B3E7F800B307FE4028
:104A800013975700635E0718370400047D147D8C6C
:104A90002285EF1060056D15B317A4006348951AC1
:104AA000058D1304150013070002018F3397E700EB
:104AB0003337E000B3D78700D98F814413F77700ED
:104AC00019C713F7F70091466303D70091071397AF
:104AD0005700635B071485041307F00F4A8663834E
:104AE000E4169A07A58313F5F40FB2402244A607F3
:104AF0009314750113D59700458D7E0692440249A3
:104B0000518D410182806399080A1387140013773D
:104B1000E70F6317071463900422630D0E1EE386EC
:104B20000EFCB307DE411397570063500722B3878B
:104B3000CE412E8961B7635C100B630E08089307A2
:104B4000F00F6383F406B7070004B3EEFE00ED47F1
:104B500063C9171F93070002B3871741B397FE007D
:104B6000B3D81E01B337F000B3E7F800F2971397FC
:104B700057006357070A85041307F00F6384E40C9A
:104B8000B706007E13D71700FD16858B758FD98F5A
:104B900035B7638D0E08FD18B307DE41E38208EEDA
:104BA0009307F00FE39DF4EA630D03080146130534
:104BB000F00FB707400015BF33079840EDE86302D8
:104BC0000E147D17630807189307F00F6319F80E8A
:104BD0002E893683D1BF638B0E04FD18B307DE0127
:104BE000E38708F89307F00FE393F4F675BF639536
:104BF0000808850413F7E40F631307126317051001
:104C0000630F0E14E3830EEEB307DE011397570014
:104C1000814463570700370700FC7D17F98F8544EF
:104C200013F77700E31F07E813D337009307F00F5C
:104C3000E38CF4F693179300A58313F5F40F4A86DB
:104C40006DB54A861305F00F814745B5370700FC5F
:104C50007D17F98F13F77700898CE31407E6E9B71E
:104C60003304DE419317540063C3070CE31204E2DC
:104C700001460145814795BD33079840ADC4930770
:104C8000F00FE308F8F4B7070004336EFE00ED47B9
:104C900063CCE70C93070002998FB317FE003357DC
:104CA000EE00B337F000D98FF697C284C9B59307E9
:104CB000F00FE30FF8F0B7070004336EFE00ED4786
:104CC00063C3E70893060002998EB316DE00B3575C
:104CD000EE003337D000D98FB387FE40C2842E89CF
:104CE00045B3854761BB630E0E067D17B307DE0132
:104CF000C284E30E07E69307F00FE31AF8F8368351
:104D000065B53683C2842E8915B7E3040EECE38DB6
:104D10000EE869BD638D0E022E86B687F9B3930740
:104D2000F00FE381F4F2B307DE018583D5BD338450
:104D3000CE412E89B1BBE31C0EFCE3890EE62E8921
:104D400049BD854725B5854741BFE39B07EC014633
:104D5000814761BBB387CE41C2842E8915B3B68724
:104D600069B33683C284D9B585473DBF397193573E
:104D700075014AD856D25ECE931A95001359F501A3
:104D800006DE22DC26DA4ED652D45AD093F7F70F3D
:104D900093DA9A00CA8B638207121307F00F6384B9
:104DA000E7128E0A37070004B3EAEA00138A17F8FD
:104DB0000144014B93D775019394950093F7F70F36
:104DC000A58093D9F501FDC71307F00F6387E702AC
:104DD0008E04938717F837070004D98C330AFA40FA
:104DE0008146558C17370000130747860A043A940A
:104DF0001C4033493901BA978287130A1AF0F9E83F
:104E00008946558C17370000130747880A043A94DF
:104E10001C4033493901BA97828701491307F00FC3
:104E2000B707400013959700F2506254931777012B
:104E300025817E095D8D33652501D2544259B259D1
:104E4000225A925A025BF24B216182801307F00FC3
:104E50008147C9BFA68ACE8B368B8947630BFB1A65
:104E60008D47E30CFBFA8547630AFB0A1307FA0731
:104E700013F91B006357E01293F77A0099C793F771
:104E8000FA0091466383D700910A93974A0063D949
:104E90000700B70700F8FD17B3FAFA0013070A086E
:104EA0009307E00FE3C4E7FA93976A00A5831377AB
:104EB000F70F8DBFB9E48546A9B763940A02114480
:104EC000014A054BC5BD63990A002144130AF00F3E
:104ED000094BCDB58D4631B73144130AF00F0D4B58
:104EE000D1BD56852EC6EF0030409307B5FFB39A6B
:104EF000FA009307A0F8338AA7400144014BB2455A
:104F000055BD2685EF00503E1307B5FFB307AA0035
:104F1000B394E400138A67078146E1B513F91B00D7
:104F20000147814701B74166139554007D16935799
:104F30000501698E63FA9A0AB3D5FA027D1AD686FC
:104F400001473388C502B3F6F602C206558F637B6C
:104F500007012A979386F5FF6368A70A6376070B14
:104F6000F9152A9733070741B356F7023377F7024B
:104F7000B38AC6029317070163FB5701AA971387E9
:104F8000F6FF63E1A70863FF5707F916AA97C20562
:104F9000B38A5741D58DB33A5001B3EA5501CA8B54
:104FA000F1B58546998E11C76D4601478147E34BA0
:104FB000D6E6130AEA09339A4A01B3D7DA00B33ABC
:104FC0004001B3E7570113F7770019C713F7F7004C
:104FD00091466303D7009107139757006348070270
:104FE0009A07A58301473DBD93D61A00B3D5F602B3
:104FF0001397FA0141833388C502B1B7CE8B368B44
:10500000814AA1BDBA8661B7B685A9BF0547814768
:1050100011BD13F91B001307F00F814721B59356FB
:105020007501B7078000FD1713D6750193F6F60FCB
:105030001308F00FB3F8A7001357F501ED8F13769F
:10504000F60FFD8163810603630C06018DE211E218
:10505000B1C3638E08026305B70405451DE782806E
:10506000F5D779558280E39E08FE6309D60211E2E6
:10507000EDD7E314B7FEE342D6FE63C7C600E3EE06
:1050800017FD0145E3FDF8FC01E77D558280F5DD64
:10509000054582800145E39208FC8280F9DBD1B7A7
:1050A0008146E1BF93567501B7078000FD1713D6FF
:1050B000750193F6F60F1308F00FB3F8A700135716
:1050C000F501ED8F1376F60FFD8163870603630903
:1050D000060185EA11EA89EB0145639B080082809D
:1050E0000945F5FFE5DA31A8638C08026300B704CF
:1050F000054575D77D55828009456398080263048C
:10510000D60211E2F5D7E315B7FEE343D6FE63C737
:10511000C600E3EF17FD0145E3F3F8FC19E3D9BF3F
:10512000F1D905458280E5D3828082808146C5B76A
:10513000797122D4135475014ECE52CC9319950037
:1051400006D626D24AD056CA5AC81374F40F93D939
:105150009900135AF50169C49307F00F6308F40E20
:105160009397390037070004B3E9E700130414F8F4
:105170008144014B13D77501939A95001377F70F6C
:1051800093DA9A0013D9F50145CF9307F00F630C1A
:10519000F7028E0A130717F8B7070004B3EAFA00FC
:1051A0003A94014633452A01BD47AA869305140067
:1051B00063E2971017270000130747518A04BA9437
:1051C0009C40BA9782871304F40F63980A0C93E407
:1051D00024000946C1BF01451307F00FB70740007F
:1051E000B2502254A6075E07A5837E05D98F92543C
:1051F0000259F249624AD24A424B5D8D4561828032
:10520000CA86D689328B89476301FB0A8D47E3043E
:10521000FBFC854736856312FB1A01478147C9B7F6
:10522000639E090413D77501939A95001377F70FBE
:1052300091440144054B93DA9A0013D9F50131F7F3
:10524000639D0A0093E414000546A9BF6393090215
:10525000A1441304F00F094B31BF5685EF00D0086D
:105260009307B5FF098CB39AFA001304A4F801461A
:1052700015BFB1441304F00F0D4BEDBD4E852EC686
:10528000EF0090069307B5FF1304A0F8B399F90057
:10529000098C8144014BB245F1BD93E434000D46C5
:1052A00011B78947D286E313FBF636851307F00F53
:1052B00081473DB741639306F3FF13D6090193D8A5
:1052C0000A01B3F7D900B3FADA0033885703B38978
:1052D000F80213570801B30A5603D6994E973306BE
:1052E0001603637357011A96C167FD17B376F7006B
:1052F0003378F800C206C296939966009357070167
:10530000B3393001E982B2979A07B3E6D900B3E91D
:10531000D7009397490063D9070013D7190093F773
:105320001900B369F7002E841307F4076350E004F3
:1053300093F7790099C793F7F90091466383D700F3
:1053400091099397490063D90700B70700F8FD1743
:10535000B3F9F900130704089307E00F63CBE704E0
:1053600093976900A5831377F70F9DBD8547B38693
:10537000E74011C76D4601478147E343D6E613076F
:10538000E4093397E9003337E000B3D7D900D98F68
:1053900013F7770019C713F7F70091466303D70097
:1053A000910713975700634C07009A07A58301479D
:1053B00005BD1307F00F814725B52E84B5B7054706
:1053C000814739BD3707800041117D17935675011C
:1053D00013D87501B377A70093F6F60F935EF50126
:1053E0003376B70026C24AC01378F80F06C622C427
:1053F0001303F00F3E8E3689F684139F3700FD812C
:1054000013153600B38806416302681093C5150072
:10541000638CBE106354100D631008106304051EE6
:10542000FD18B307AF40638608029307F00F638847
:10543000F616ED4763C71729130700023307174114
:105440003317E500B35715013337E000D98FB307A1
:10545000FF40139757006351071A370400047D1467
:105460007D8C228551256D15B317A400634E251B35
:10547000330525411304150013070002018F3397EC
:10548000E7003337E000B3D78700D98F014913F71E
:10549000770019C713F7F70091466303D700910708
:1054A00013975700635E0714930619001307F00F54
:1054B00093FE14006386E6169A07A58393F6F60F0B
:1054C000A607B240224413D59700DE069397FE014B
:1054D000558D924402495D8D410182806392080A94
:1054E000138716001377E70F631B071463940622D4
:1054F00063020F2071D5B307AF4013975700635570
:105500000722B307E5410149AE8451B7E30005F036
:10551000638ABE0AE35410FD9307F00F6381F60817
:10552000B70700045D8D31B7635E10096301080899
:105530009307F00F6385F606B70700045D8DED470E
:1055400063C0171F13070002330717413317E50025
:10555000B35715013337E000D98FFA9713975700E7
:10556000635C070805091307F00F630BE90AB70628
:10557000007E13D71700FD16858B758FD98F01BF5D
:105580003307D84063950610630D0F147D1763032E
:10559000071A9307F00F6314F810AE84328E630F6E
:1055A0000E06814E9306F00FB707400011BF39C9B0
:1055B000FD18B307AF00E38308FA9307F00FE390F9
:1055C000F6F8F1BF63990808138916001377E90FFD
:1055D00063160712639B061063030F16E30205EEC2
:1055E000B307AF0013975700014963570700370708
:1055F00000FC7D17F98F054913F77700E31C07E8D6
:1056000013DE37009307F00FE30BF9F893179E00B2
:10561000A5839376F90F93FE14005DB593FE1400F5
:105620009306F00F814769BD370700FC7D17F98F9E
:1056300013F777003309A940E31E07E4D1B7330419
:10564000AF409317540063C3070CE31C04E0814E82
:1056500081468147B5B53307D840B5C69307F00FEB
:10566000E30EF8F2B7070004336FFF00ED4763CD98
:10567000E70C93070002998FB317FF003357EF0031
:10568000B337F0005D8FB307A7004289C1BD930710
:10569000F00FE304F8F0B7070004336FFF00ED47A5
:1056A00063C2E70893070002998FB317FF003357CF
:1056B000EF00B337F000D98FB307F5404289AE84CD
:1056C00049BB854769B3630E0F067D17B307AF006B
:1056D0004289E30507E89307F00FE319F8F8328EE3
:1056E0007DBD328E4289AE8431BFE3090FEAE30803
:1056F00005EA45BD0DCDAE8EB287D9B39307F00F45
:10570000E300F9F2B307AF008583FDB53304E5414B
:10571000AE8481BBE31D0FFCE30505E8AE84BDBD8F
:10572000854725BD854749BF0149E39707EC814E71
:10573000814779B3B307E5414289AE8419BBB2878B
:1057400041B3328E42897DBD054735BF37068000A3
:10575000135775019307F6FF1377F70F9305E007CB
:10576000B3F6A7009357F50163FCE5009305D00954
:1057700063FAE500370500801345F5FF3E9582800A
:105780000145828093055009D18E63CDE500130653
:1057900060093307E64033D7E6003305E040F5F310
:1057A0003A8582801307A7F63397E600FDB71357B3
:1057B0007501370680009307F6FF1377F70F9305FF
:1057C000E007B3F6A7009357F501014563F4E50040
:1057D00099C3828082809307E0097D55E3EBE7FE61
:1057E00093055009B3E7C60063D7E5001307A7F692
:1057F0003395E7008280130560093307E54033D510
:10580000E7008280411106C622C415CD2A84E92C06
:105810009307E0093387A7409307600963C0E70453
:10582000A1469377F70F63D5A60061153314A40042
:1058300026042580260413559400B2402244DE0736
:105840005D8D410182800144260413559400B240CD
:1058500022448147DE075D8D4101828093079009D4
:1058600063DDE7009307B5019546B317F400898E11
:10587000B337F0003354D4005D8C954763D6A7004E
:105880009307B5FF3314F400B70600FCFD169377B9
:1058900074003376D40085C39377F4009145638C0C
:1058A000B70011069317560063D707009307F00956
:1058B000758E3387A7401314660025802604135580
:1058C0009400B24022449377F70FDE075D8D4101CB
:1058D0008280135775011377F70F41119307170053
:1058E00022C426C21314950006C693F7E70F25803D
:1058F0009354F50185C7935734001307073876048E
:10590000B2075207B1831395F401D98FC98FB24002
:10591000228522449244BE854101828005EB39C430
:105920002285D922A94763C6A7042D47098F93076B
:1059300055013357E4003314F4009317C7001307DD
:105940009038098FB1831377F77F5DBF01CC135770
:105950003400B7070800D98FB2077604B183130764
:10596000F07F79BF1307F07F814759BF0147814717
:1059700041BF130755FF3317E40001447DBF93D6A1
:1059800045019397C50093F6F67FB1831386160001
:105990008E071357D5011376E67FFD815D8F93182F
:1059A000350035CE138806C89307E00F63DD070185
:1059B0008147139597009306F00FDE062581FE05BB
:1059C000558D4D8D82806355000B931765000E0732
:1059D000B337F000D98F93D8D801B3E7170113F785
:1059E00077006301071013F7F70091466303D700B0
:1059F0009107370700047D8F75C71307180013063A
:105A0000F00F9376F70FE305C7FA9A07A58313956E
:105A10009700DE062581FE05558D4D8D8280B3678A
:105A2000170199EE85CF95479A07A583139597009F
:105A300093F6F60FDE062581FE05558D4D8D82808D
:105A4000A5DBB7074000139597009306F00FDE061D
:105A500081452581FE05558D4D8D828081471395A9
:105A600097008146DE062581FE05558D4D8D82808D
:105A7000A5576348F804F94737068000B387074104
:105A80007D45598E6351F504795733070741130556
:105A900000023357E6006388A700938626CAB31630
:105AA000D600B3E8D800B3371001D98F13F77700C9
:105AB000014815FB139757008546E34807F48146D4
:105AC000A5B781468DB7938626C83397D80033375C
:105AD000E000B316D600B3D8F800B367D700B3E739
:105AE000F800E9B7C28689B7C167637CF5029307FE
:105AF000F00F1307000263EBA700972700009387BE
:105B0000E7C0AA9788233305A74082802181972781
:105B100000009387A7BFAA97882361473305A74052
:105B20008280B7070001636DF5006181972700004F
:105B30009387C7BDAA97882321473305A740828052
:105B4000418197270000938767BCAA978823414724
:105B50003305A7408280B3C7A5008D8B3307C500EE
:105B600081E78D4763EDC700AA87637EE50894212E
:105B700085078505A38FD7FEE3EBE7FE828093764A
:105B80003500AA8789CA942185078505A38FD7FE8A
:105B900093F63700C5BF9376C7FF138606FE63F002
:105BA000C70683A3050083A2450083AF850003AF2A
:105BB000C50083AE050103AE450103A3850183A89B
:105BC000C5019385450223A0770003A8C5FF23A242
:105BD000570023A4F70123A6E70123A8D70123AA8E
:105BE000C70123AC670023AE17019387470223AE9A
:105BF00007FF75B790419107910523AEC7FEE3EB10
:105C0000D7FEE3E6E7F6828039713EDA2ED232D44F
:105C100036D63AD842DC46DE9387818122CC804357
:105C200026CA06CEAA8409C41C4C99E32285E12B1E
:105C30000C4454102686228536C6EF00D021F2404F
:105C40006244D24421618280011126CA4AC806CE2C
:105C500022CC4EC652C4AA842E8901C51C4D91E3A4
:105C60005D239C4C804499E32685712B9727000087
:105C70009387C7BB631BF402C0405E24A18BB1C7EE
:105C80001C48A1C7FD59294A1C4483450900FD173A
:105C9000B1E91CC463DD07062286A9452685952245
:105CA000FD576308F502294535A097270000938723
:105CB000E7B96314F4008044C9B7972700009387BD
:105CC000E7B4E31CF4FAC0444DBFA2852685C52A7B
:105CD00055D97D55F2406244D2444249B249224AE4
:105CE000056182801CC4050963D70700184C63CA8C
:105CF000E700638845011C401387170018C08CA378
:105D000061B722862685F528E31035F9D9B71C40FE
:105D10001387170018C0294798A371B7938781810B
:105D2000AA8588436FF05FF241119387818122C475
:105D3000804326C206C61C5CAA848DEB61452527DC
:105D4000B737CDAB08DC9387E7301CC1B7176DE6DA
:105D5000938747235CC1B7E705009387C7EE1CC54F
:105D6000AD475EA50547814718C95CC91C5CB240B8
:105D7000224484CB23AA070092444101828041112E
:105D80009387818122C4804306C61C5C8DEB6145EC
:105D9000D92DB737CDAB08DC9387E7301CC1B717D7
:105DA0006DE6938747235CC1B7E705009387C7EE8D
:105DB0001CC5AD475EA50547814718C95CC9105C85
:105DC0003787954CB7F75158144A484A1307D7F20A
:105DD0009387D742B387F602B24022443305E502E7
:105DE0003E95B387E60233B7E6029386170014CADE
:105DF0002A9733B5F6003A9548CA06050581410150
:105E00008280011122CC26CA4AC806CE4EC6AA8478
:105E10002E89328401C51C4D91E3F5269727000099
:105E20009387C7A06317F406C0401C4C1CC45E24B3
:105E3000A18BC1C31C48B5CF1C4808409379F90F0A
:105E40001379F90F1D8D5C486346F500A285268500
:105E5000692C25E51C440505FD171CC41C4013874F
:105E6000170018C0238037015C486388A7005E24B0
:105E7000858B81CBA9476316F900A2852685B524B9
:105E80000DEDF24062444A85D2444249B24905616F
:105E90008280972700009387679B6314F4008044F7
:105EA00069B79727000093876796E310F4F8C0441A
:105EB000ADBFA2852685212041D17D59D9B7411199
:105EC0009387818126C2844322C44AC006C62A8998
:105ED0002E8489C49C4C99E326853526972700009B
:105EE0009387C794631BF402C0400317C400931741
:105EF0000701C18393F68700ADEA93F6070195EE9B
:105F0000A5472320F900136707045AA47D55B24022
:105F100022449244024941018280972700009387DE
:105F2000E7926314F4008044C9B797270000938771
:105F3000E78DE31CF4FAC0444DBF918B9DC34C58D0
:105F400089C9930744046384F5004A851523232AED
:105F500004025E242322040093F7B7FD5EA41C48CC
:105F60001CC05E2493E787005EA41C4899EB5E2466
:105F70001307002093F707286385E700A2854A8569
:105F800091295E2413F717001DC35C4823240400E5
:105F9000B307F0401CCC1C480145B5FB8317C40077
:105FA00013F707082DD793E707045EA485B7898BFD
:105FB000014791E3584818C4F9BFDE25011122CCEE
:105FC00026CA06CE4AC84EC613F78700AA842E8476
:105FD00079EBD841634DE000B841634AE0000145E8
:105FE000F2406244D2444249B24905618280585429
:105FF0007DD703A904009396370123A0040063DB37
:10600000060670485E24918B99C75C401D8E5C58D3
:1060100099C33C401D8E5C540C5081462685829766
:10602000FD575A24631DF5009440F54763E8D706F1
:10603000B70740208507B3D7D700858BA5C31C4879
:10604000232204001CC09317370163D80700FD57B3
:106050006314F5009C4091E368C84C5823A02401C8
:10606000BDDD930744046384F50026851121232AAE
:106070000402B5B70C500146854626850297FD57A8
:106080002A86E311F5F89C40B5DF75476385E70084
:1060900059476393E70423A0240191B713670704CA
:1060A0005AA47D5535BF83A90501E38A09F203A9E6
:1060B00005008D8B23A0350133093941014791E358
:1060C000D84918C4E35D20F11C540C50CA864E8692
:1060D000268582976347A0005E2493E707045EA4A9
:1060E000C9B7AA993309A940F1BF9C49A5C30111B9
:1060F00022CC06CE2A8411C51C4D81E72EC6212252
:10610000B2459717000093876772639CF5004C4077
:106110008397C5009DC722856244F24005616FF0F8
:10612000DFE997170000938767726394F5000C44CA
:10613000C5B7971700009387676DE39BF5FC4C4448
:10614000C1BFF24062440145056182800145828001
:10615000411122C406C62A844EA572A5232005003B
:1061600023220500232405002322050623280500F9
:10617000232A0500232C0500214681451305C5056A
:10618000EFA00F8297170000938727B35CD0971773
:106190000000938747B51CD497170000938727B951
:1061A0005CD497170000938787BB00D01CD8B240FF
:1061B00022444101828097050000938545F391AA0E
:1061C000411126C2130680069384F5FFB384C402EE
:1061D0004AC02E8922C406C693854407352E2A84D8
:1061E00001CD2320050023222501310508C4138693
:1061F00084068145EF90DFFA2285B2402244924422
:106200000249410182801C4DA5E7411106C622C406
:1062100097070000938767FA1CD59387C1819C4339
:106220002324050423260504232805046314F5000C
:1062300085471CCD2A84352848C022851D2808C4DE
:106240002285052848C4484001469145EFF05FF09B
:1062500008440546A545EFF0BFEF48440946C94547
:10626000EFF01FEF85471CCCB240224441018280F1
:10627000828041119387C18126C284434AC006C6E9
:106280009C4C22C42A8981E72685EFF0DFF79384AE
:1062900084048044DC40FD1763D607009C40B9CFDE
:1062A0008440C5BF0317C40039E7C177850723229F
:1062B00004062320040023220400232404005CC4D9
:1062C00023280400232A0400232C040021468145AE
:1062D0001305C405EF90DFEC232A0402232C0402EB
:1062E00023240404232604042285B2402244924439
:1062F0000249410182801304840671BF91454A8599
:10630000EFF01FEC88C049FDB1472320F90001449C
:10631000E1BF797122D44AD052CC56CA5AC85EC65F
:1063200006D626D24ECE2A8AAE8A130485040149A7
:10633000054BFD5B09ECB25022544A859254025938
:10634000F249624AD24A424BB24B456182800444D0
:1063500083294400FD1963D409000040E1BFDE2415
:10636000637BFB008397E40063877701A6855285F2
:10637000829A3369A90093848406E9BF1971A6DA69
:10638000AE848395E500A2DC86DE328463DB050003
:10639000DE2423A0060093F7070885E79307004053
:1063A0001DA0300836C6EF001021B246E34205FEBC
:1063B0007247BD67F98F7977BA9793B717009CC278
:1063C000F1BF930700041CC0F6506654D654014533
:1063D00009618280DE25011122CC06CE26CA4AC878
:1063E000898B2E8489CF930774041CC01CC88547F1
:1063F0005CC8F2406244D244424905618280740024
:106400003000AA84EFF09FF7A2452A892685292229
:1064100019E98317C40013F7072061FFF19B93E785
:1064200027005EA4C9B797070000938707D99CD4BB
:106430005E2408C008C893E707085EA4A2475CC8AA
:10644000B24781CF8315E4002685EF00701911C58E
:106450005E24F19B93E717005EA45E243369F90084
:106460002316240179B793878181AA8588436DA07B
:10647000DDC183A7C5FF411122C406C626C213840D
:10648000C5FF63D307003E94AA84EF00301C9387B6
:10649000C1889C4381EF2322040023A681882244E3
:1064A000B2402685924441016F00701A637EF40069
:1064B00014403307D4006396E7009843DC433697D3
:1064C00018C05CC0D9BFBA87D84319C3E37DE4FEC6
:1064D00094433386D700631F86001040B29694C35E
:1064E0003386D700E31DC7FA10435843B29694C3CE
:1064F000D8C375B76375C400B1479CC04DB7104091
:10650000B306C4006316D70014435843B29614C0B0
:1065100058C0C0C369B78280011126CA9384350070
:10652000F19806CE22CC4AC84EC6A104B14763F307
:10653000F404B14463E2B4042A89EF003011938774
:10654000C18898433A8439E0938701899C4391E755
:1065500081454A85252F23A8A188A6854A853D2700
:10656000FD5963193507B1472320F9004A85EF002B
:10657000100E29A0E3D004FCB1471CC10145F24034
:106580006244D2444249B249056182801C40858FF1
:1065900063CF0702AD4663F6F6001CC03E9404C00C
:1065A00031A05C406313870223A6F1884A85EF007F
:1065B000100A1305B4009307440061993307F540AE
:1065C0005DDF3A94898F1CC05DBF5CC3C5B722876D
:1065D000404095BF130435007198E30285FCB30574
:1065E000A4404A856525E31C35FBB5BF1C46FD1755
:1065F0001CC663DA0700184E63C5E700A947639419
:10660000F5006FF01F801C422E851387170018C2FB
:106610008CA38280011122CC26CA4AC84EC652C41D
:1066200006CE2A89AE893284B304D6007D5A63141B
:106630009400014509A80C204E864A85EFF01FFB07
:106640000504E31645FFF2406244D2444249B24990
:10665000224A05618280357122CD26CB4AC94EC7B8
:1066600006CF52C556C35AC1DEDEE2DCE6DAAA899D
:10667000AE843289368409C51C4D99E3EFF0BFB86A
:10668000971700009387871A6398F40C83A4490036
:10669000DE24A18BE5C79C48F5C393070002A30441
:1066A000F1029307000302D22305F10222C6930BE5
:1066B0005002971A0000938A6A1B054C294B4A84A2
:1066C0001C2099C3639F770DB30C2441638E0C008B
:1066D000E6864A86A6854E85EFF0DFF3FD57630F09
:1066E000F51C9256E69636D21C206389071CFD578E
:1066F0001309140002C802CE3ECA02CCA309010449
:1067000082D483450900154656852D2713041900A8
:10671000C24751E913F7070109C713070002A3098C
:10672000E10413F7870009C71307B002A309E104C6
:10673000834609001307A002638FE606F2474A84E6
:1067400081462546182093051400130707FD63773B
:10675000E60AB5CA3ECE85A8971700009387070FB3
:106760006395F40083A4890025B7971700009387E9
:10677000E709E39FF4F083A4C90019BFA6854E85FD
:10678000EFF0EFF319D97D55FA406A44DA444A49EB
:10679000BA492A4A9A4A0A4BF65B665CD65C0D6196
:1067A0008280050431BF330555413315AC00C98FD4
:1067B0003EC82289B9B7324793064700184336C608
:1067C000634707023ACE18209307E002631DF704DF
:1067D00018309307A002631BF702B247090413871E
:1067E00047009C433AC663C107023ECA2DA833073F
:1067F000E04093E727003ACE3EC8F1B7B38767037E
:1068000085462E84BA973DBFFD57C5B7050402CA19
:10681000814681472546182093051400130707FD7C
:106820006374E606F9F20C200D46171500001305F7
:106830006504092511CD971700009387A7031D8DC7
:1068400093070004B397A700424505045D8D2AC84D
:106850000C20194617150000130505021309140032
:106860002304B102C12B35C19797FFFF9387877926
:1068700095E74247B2471377071009CF91073EC605
:106880009257D2973ED225BDB387670385462E84A3
:10689000BA9751B79D07E19BA107D5B77800970636
:1068A0000000938666D726860C084E859700000068
:1068B000E7000000FD572A8AE314F5FCDE2493F775
:1068C0000704E39207EC1255C1B578009706000063
:1068D000938686D426860C084E85012AE1BF7971FD
:1068E00056CA9C49BA8A984522D426D24ECE52CC5A
:1068F00006D64AD05AC85EC6AA892E84B284368A81
:1069000063D3E700BA879CC00347340419C38507E3
:106910009CC01C4093F7070281C79C4089079CC01C
:106920000329040013796900631A0900130B940109
:10693000FD5B5C449840998F634CF9041C4083468E
:10694000340493F70702B336D000A5EB13063404E2
:10695000D2854E85829AFD576303F5041C4011468B
:106960009840998B544481446397C700B384E640B0
:1069700063D3040081441C4418486354F700998F82
:10698000BE94014969047D5B63982405014509A80B
:1069900085465A86D2854E85829A631E75017D553D
:1069A000B250225492540259F249624AD24A424B9E
:1069B000B24B456182800509ADBF3307D400130691
:1069C0000003A301C7040347540493871600A2974A
:1069D0008906A381E7049DBF85462286D2854E8520
:1069E000829AE30E65FB050945B7797122D426D258
:1069F0004AD04ECE06D652CC56CA5AC8B689942D25
:106A0000930790063289AA842E8413863504638DF9
:106A1000F60263E2D706930780056386F61863EDF6
:106A2000D700638E062093073004638EF60A930A1C
:106A300024042301D404C9A0930730066385F60A11
:106A400093074006E395F6FE1C40084393F60708BB
:106A500093054500C5C61C410CC363D80700130746
:106A6000D002B307F040A301E40497160000938618
:106A700026E1294765A8930700076382F61663E5B8
:106A8000D7029307E0066389F6189307F006E390B0
:106A9000F6FA0C401C4313F80508138547006307FA
:106AA000080608C39C4385A893075007E383F6FEB6
:106AB000930780076389F61293073007E399F6F688
:106AC0001C43D04181459386470014C383AA070025
:106AD00056858D2601C53305554148C05C401CC80C
:106AE000A301040461A81C43930A2404938647006D
:106AF0009C4314C32301F4048547D5B793F60704D8
:106B00001C410CC3B9DAC207C18781BF93F50504E4
:106B100008C3C9D99E231307F0066387E60E9716AC
:106B200000009386E6D52947A30104044C400CC419
:106B300063C5050008406D9908C099E3B28A89CD04
:106B4000B28AB3F5E702FD1AB6958C212380BA000C
:106B5000B3D5E70263F0E70CA147631EF7001C40C2
:106B6000858B91CB58401C4863C7E700930700030F
:106B7000A38FFAFEFD1A3306564110C84E87CA8607
:106B80007000A2852685EFF09FD57D5A631D450BC9
:106B90007D55B250225492540259F249624AD24A67
:106BA000424B45618280A382D504971600009386EC
:106BB00026CD0C40084313F805081C411105630D50
:106BC000080208C313F7150001C793E505020CC0BE
:106BD0004147B9FB0C4093F5F5FD0CC0B1B79C41A2
:106BE00093E707029CC193078007A302F40497165A
:106BF0000000938626CA75BF13F8050408C3E30393
:106C000008FCC207C1837DBF97160000938646C764
:106C1000214719BFAE8735B794411C43CC4913F8BF
:106C20000608138547006306080008C39C438CC30D
:106C300039A008C393F606049C43F5DA8EA32328F3
:106C40000400B28A25BF14485686CA8526858299D3
:106C5000E30045F51C40898B8DE7B2474844E35A71
:106C6000F5F23E853DB785465686CA8526858299CA
:106C7000E30065F3050A5C443247998FE345FAFE69
:106C8000E9BF014A930A94017D5BF5B7411122C423
:106C90002A842E8523AA01B406C6EFA0FFE6FD577D
:106CA0006317F500938741B59C4391C31CC0B24064
:106CB000224441018280411122C42E848395E50043
:106CC00006C67922634905007C48AA977CC8B24071
:106CD0002244410182805E247D777D17F98F5EA476
:106CE000FDB7DE25011122CC26CA4AC84EC606CE03
:106CF00093F70710AA842E843289B68991C78395A9
:106D0000E5008946014609225E247D777D17F98FCB
:106D10005EA48315E4006244F240CE864A86B249FE
:106D200042492685D244056125A8411122C42E84FA
:106D30008395E50006C6C928FD575A24631AF50055
:106D4000FD77FD17F98F5EA4B24022444101828095
:106D50008567D98F5EA468C8C5BF8395E50005A87F
:106D6000411122C42A842E85B285368623AA01B415
:106D700006C6EFA09FD5FD576317F500938741B571
:106D80009C4391C31CC0B240224441018280411106
:106D900022C42A842E8523AA01B406C6C520FD5725
:106DA0006317F500938741B59C4391C31CC0B24063
:106DB000224441018280411122C42A842E85B28559
:106DC00023AA01B406C6C920FD576317F5009387AF
:106DD00041B59C4391C31CC0B24022444101828012
:106DE000411122C42A842E8523AA01B406C65D203F
:106DF000FD576317F500938741B59C4391C31CC0B1
:106E0000B240224441018280411122C42A842E854D
:106E1000B285368623AA01B406C65920FD576317EA
:106E2000F500938741B59C4391C31CC0B2402244F6
:106E30004101828093F5F50F2A966314C500014540
:106E400082801C21E38EB7FE0505C5BF828082804B
:106E5000411122C42A842E85B285368623AA01B424
:106E600006C6A920FD576317F500938741B59C43DB
:106E700091C31CC0B2402244410182809307800527
:106E800023AAF1B47D5582809307800523AAF1B42B
:106E90007D5582809307800523AAF1B40145828045
:106EA0009307800523AAF1B47D558280930780055E
:106EB00023AAF1B47D55828053797374656D436C58
:106EC0006B3A25640D0A00004368697049443A250D
:106ED0003038780D0A00000043616C696272617499
:106EE00074696F6E5F56616C203A2025640A000059
:106EF0000000003F6666663F0000F04300000000AF
:106F0000CDCCCCCCCCCCEC3F696E2074696D3120FB
:106F1000697271200000000000F07F450000000051
:106F20006666666666660A40000000000000104063
:106F3000000000000000E03F0000000000003440BE
:106F400000000000000026407B0E710E670E5C0EF4
:106F5000510E460E3B0E300E240E180E0C0E000E77
:106F6000F30DE70DDA0DCD0DBF0DB20DA40D960D8D
:106F7000880D790D6A0D5B0D4C0D3D0D2D0D1E0D0F
:106F80000D0DFD0CED0CDC0CCB0CBA0CA90C970C08
:106F9000850C730C610C4F0C3C0C2A0C170C030C69
:106FA000F00BDD0BC90BB50BA10B8D0B780B640B34
:106FB0004F0B3A0B260B100BFB0AE60AD00ABB0A52
:106FC000A50A8F0A790A630A4D0A370A200A0A0AB3
:106FD000F409DD09C709B009990983096C09550944
:106FE0003E0927091109FA08E308CC08B5089F08EB
:106FF000880871085A0844082D0817080008EA078D
:10700000D307BD07A70791077A0765074F07390719
:1070100023070E07F806E306CE06B906A4068F0678
:107020007A06660651063D06290615060106EE0596
:10703000DA05C705B405A1058E057B05690556056A
:107040004405320520050F05FD04EC04DB04CA04E9
:10705000B904A8049804880478046804580449040E
:1070600039042A041B040C04FE03EF03E103D303D9
:10707000C503B703AA039C038F0382037503680348
:107080005C035003430337032B032003140309035A
:10709000FD02F202E702DC02D202C702BD02B30225
:1070A000A9029F0295028B02820278026F02660299
:1070B0005D0254024C0243023B0232022A022202C7
:1070C0001A0212020A020302FB01F401ED01E601B9
:1070D000DE01D701D101CA01C301BD01B601B00172
:1070E000AA01A4019E01980192018C0186018101EF
:1070F0007B01760170016B01660161015C01570142
:1071000052014D01480144013F013B01360132016A
:107110002D012901250121011D011901150111016F
:107120000D010A0106010201FF000000381F0000E6
:10713000461F0000521F00005E1F0000C01F00001D
:1071400000401C460000C842000000400000904182
:107150000000684100000000333333333333D33F42
:107160000000C040000080419A9999999999A93FDF
:10717000B81E85EB51B89E3F9A9999999999D93F34
:107180009A9999999999B93F17B75138ACC527374A
:107190006F12033ABD37863500007A440AD7A33B05
:1071A0005B494E464F5D205B25733A25645D205256
:1071B0006567697374726174696F6E207375636358
:1071C000657373200D0A0D0A000000005B455252E2
:1071D0004F525D205B25733A25645D202052656720
:1071E00069737465725F4E756D6265722065727247
:1071F0006F723A2578200D0A0D0A00005B45525245
:107200004F525D205B25733A25645D2020526567EF
:1072100069737465725F53746172745F4164647200
:10722000657373206572726F72203A202578200D85
:107230000A0D0A00696E20777269746520726567AD
:1072400069737465722000005B494E464F5D205B98
:1072500025733A25645D2020534C5F52656164526A
:107260006567697374657242617474657279566F8B
:107270006C74616765200D0A000000005B494E4692
:107280004F5D205B25733A25645D2020534C5F528F
:10729000656164526567697374657243686172679A
:1072A00043757272656E74200D0A00005B494E468C
:1072B0004F5D205B25733A25645D2020534C5F525F
:1072C0006561645265676973746572446973636864
:1072D00061726743757272656E74200D0A0000005A
:1072E0005B494E464F5D205B25733A25645D202047
:1072F000534C5F526561645265676973746572448B
:10730000697363686172674D6F735374617465204C
:107310000D0A0000000020415B494E464F5D205B96
:1073200025733A25645D2020534C5F526561645299
:107330006567697374657248696768536964654D08
:107340006F7354656D7065726174757265200D0A96
:10735000000000005B494E464F5D205B25733A25D7
:10736000645D2020534C5F526561645265676973A8
:107370007465724D5050544D6F6465200D0A0000C5
:107380005B494E464F5D205B25733A25645D2020A6
:10739000534C5F52656164526567697374657253DB
:1073A0006F6C61724F70656E436972637569745674
:1073B0006F6C74616765200D0A0000005B494E46E2
:1073C0004F5D205B25733A25645D204D61746368D1
:1073D0005F5374617274666C616720737563636573
:1073E0007373200D0A0D0A005B494E464F5D205B0A
:1073F00025733A25645D204D617463685F61646440
:10740000726573732073756363657373200D0A0D62
:107410000A0000005B494E464F5D205B25733A250C
:10742000645D204D617463685F42726F6164636183
:1074300073746164647265737320737563636573D9
:10744000730D0A0D0A0000005B494E464F5D205B3C
:1074500025733A25645D20526561645F52656769F2
:10746000737465720D0A0D0A000000005B494E46F8
:107470004F5D205B25733A25645D20577269746502
:107480005F52656769737465720D0A0D0A0000002A
:107490005B494E464F5D205B25733A25645D204F66
:1074A00074686572206672616D65730D0A0D0A005D
:1074B0005B494E464F5D205B25733A25645D204253
:1074C000726F6164636173745F5363616E0D0A0D63
:1074D0000A0000005B494E464F5D205B25733A254C
:1074E000645D20526567697374726174696F6E5F61
:1074F000726571756573740D0A0D0A005B494E461D
:107500004F5D205B25733A25645D2066756E636F61
:107510006465206572726F722025780D0A0D0A006D
:1075200020647574795F726174696F203A202564F4
:107530002F31303030200A0020766F7574203A20C9
:1075400025642F313030200A0000000020496F757B
:1075500074203A2025642F313030200A00000000CA
:1075600020496469736F7574203A2025642F313087
:1075700030200A00206D6F7354203A2025642F318B
:1075800030200A00206D6F735374617465203A20B7
:107590002564200A0000000020302EC3BBD3D0B9E0
:1075A000A4D7F73B20312EE4B8C1F7C4A3CABD3B32
:1075B00020322EBAE3C1F7C4A3CABD3B20332EBA92
:1075C000E3D1B9C4A3CABD3B20342EB8A1B3E4C4EF
:1075D000A3CABD3B20352EC3BBD3D0B5E7B3D8205B
:1075E0003A202564200A00007B14AE47E17A843FEC
:1075F000766F6C7420696E203A2025642F3130300C
:10760000200A00003333333FA2C9FFFF94C8FFFFB5
:1076100094C8FFFF92C8FFFF9AC8FFFF9AC8FFFFF8
:1076200060C8FFFF92C8FFFF9AC8FFFF60C8FFFF56
:107630009AC8FFFF92C8FFFF8EC9FFFF8EC9FFFFE8
:107640008EC9FFFF60C8FFFFDED8FFFF04D8FFFF31
:10765000D8D8FFFF0CD8FFFFD8D8FFFFD2D7FFFF45
:10766000D8D8FFFF0CD8FFFF04D8FFFF04D8FFFFD6
:10767000D2D7FFFF0CD8FFFF12D8FFFF12D8FFFFB1
:1076800012D8FFFFD2D7FFFFC4D7FFFFC4D7FFFF39
:1076900098D8FFFF74D9FFFF98D8FFFF92D7FFFF5C
:1076A00098D8FFFF74D9FFFFC4D7FFFFC4D7FFFFEF
:1076B00092D7FFFF74D9FFFFD2D7FFFFD2D7FFFFCA
:1076C000D2D7FFFF92D7FFFFECDBFFFF3ADBFFFFD4
:1076D0003ADBFFFF38DBFFFF3EDBFFFF3EDBFFFF58
:1076E0000EDBFFFF38DBFFFF3EDBFFFF0EDBFFFFA4
:1076F0003EDBFFFF38DBFFFFDADBFFFFDADBFFFFFC
:10770000DADBFFFF0EDBFFFF0001020203030303CE
:107710000404040404040404050505050505050521
:107720000505050505050505060606060606060601
:1077300006060606060606060606060606060606E9
:1077400006060606060606060707070707070707D1
:1077500007070707070707070707070707070707B9
:1077600007070707070707070707070707070707A9
:107770000707070707070707070707070707070799
:107780000707070707070707080808080808080881
:107790000808080808080808080808080808080869
:1077A0000808080808080808080808080808080859
:1077B0000808080808080808080808080808080849
:1077C0000808080808080808080808080808080839
:1077D0000808080808080808080808080808080829
:1077E0000808080808080808080808080808080819
:1077F0000808080808080808080808080808080809
:107800000808080808080808000000000000000038
:107810000000000000000000000000000000000068
:107820000000000000000000000000000000000058
:107830000000000000000000000000000000000048
:107840000000000000000000000000000000000038
:107850000000000000000000000000000000000028
:107860000000000000000000232D302B200000004D
:10787000686C4C006566674546470000303132331E
:10788000343536373839414243444546000000001C
:107890003031323334353637383961626364656686
:0478A00000000000E4
:1078A40000000000000000000102030406070809AC
:1078B4000000000001020304010203040607080992
:1078C40000000000000000000000000000E8037851
:1078D400050A00A406DC05B0040A000A0001000140
:1078E400001400460032002800000000534C11111F
:1078F40011111111110100010016000030000000E7
:10790400F4270000100000007E250000A000000005
:107914004A250000A1000000FA240000D000000065
:1079240056270000D1000000B82600000001000026
:10793400BE240000010100008224000002010000B6
:1079440046240000030100000A2400000401000092
:10795400CC23000005010000A8230000060100005C
:107964007E230000000000000300000080250000CA
:107974000000000000000000000000000000000003
:10798400000000000400000080250000000000004A
:1079940000000000000000000000000000000000E3
:1079A40028780000487800000878000000000000F3
:1079B40000000000000000000000000000000000C3
:1079C40000000000000000000000000000000000B3
:1079D40000000000000000000000000000000000A3
:1079E4000000000000000000000000000000000093
:1079F4000000000000000000000000000000000083
:107A0400006CDC0202040608B80400203333333F60
:107A14000101010101000000FC000020FC00002025
:00000001FF
